:0400000057EF00F0C6
:100008002B002B002B002B002B002B002B002B0090
:10001800E35B2B002B002B002B002B002B002B006D
:100028002B002B002B002B002B002B002B002B0070
:100038002B002B002B00B4562B002B002B008F5BC2
:100048002B002B00C75A2B002B002B002B002B005A
:100058002B002B002B002B002B002B002B002B0040
:100068002B002B002B002B002B002B002B002B0030
:100078002B002B002B002B002B002B002B002B0020
:100088002B002B002B002B002B002B002B002B0010
:100098002B002B002B002B002B002B002B002B0000
:0A00A8002B002B00FF00C4EFABF0AB
:10F506000000000000001B1B0000181818181B1B29
:10F516000000030303031B1B00001B1B1B1B1B1B01
:10F5260000040E1F0404040400040404041F0E0453
:10F53600001F1F1F1F1F1F1F000E0A0E00000000C6
:10F5460000DA6F01A46C01F26E01E24A01705B0100
:10F55600CA5E012A5A01CC6F017870017470017E6F
:10F566006D01207001287001BE6F01187001AE6F29
:10F5760001F06201B460019E6F010024744C002406
:10F58600744C0000FA460024F4480000FA46008055
:10F59600C094D43F35864020417574726573203A15
:10F5A60020204C43445F34626974735F4932435F81
:10F5B600323032352D30322E682C55415254315F5F
:10F5C60046756E6374696F6E732E68202C4C4344C7
:10F5D6005F63686172735F53706563696175785FB5
:10F5E600323032352D30322E680D0A0D0A00204495
:10F5F60069726563746F7279203A433A5C4D504C78
:10F606004142585F50726F6A656374735C5F31384C
:10F616004632374B34325F494E413232365F4932D9
:10F62600435F4C43445F554152545F323032352E6E
:10F63600580D0A0045434F2E2E2E2E00424152529F
:10F64600455F470042415252455F44004241525293
:10F6560045474400464C454348204800464C4543F0
:10F66600485F42004E4F49522E2E2E0044454752C7
:10F676004543200020524131206C6967687420623E
:10F6860061727269657220205241343D6C65642056
:10F69600205241333D5351412C5243363D5458205C
:10F6A6005541525431205243373D5258205541520C
:10F6B600540D0A0020496E636C7564653A204469EE
:10F6C600616C6F6775655F4F7065726174657572A1
:10F6D6005F50435F7669615F554152545F32303205
:10F6E600352D30322E696E630D0A00204C434420BE
:10F6F60034783230206361727320737572206275BC
:10F70600732049324331204857203A205243333D33
:10F7160053434C2C5243343D5344410D0A00205070
:10F72600726F6A656374203A20205F31384632373B
:10F736004B34325F4932435F4C435F554152545F0D
:10F74600323032330D0A00205049433138463237C1
:10F756004B3432202B20494E413232362052313042
:10F7660030204932432073656E736F72200D0A0094
:10F7760020436F6E6669672020496E7465726E61FC
:10F786006C20466F73632036344D487A0D0A00208C
:10F79600536F75726365203A20206D61696E2E6322
:10F7A600205F323032352D303232340D0A002020BF
:10F7B6004D46494E544F53432028353030206B4830
:10F7C6007A2900204D46494E544F53432F34202862
:10F7D6003332206B487A2900202020202020202048
:10F7E60020202020202020202020202000204565C9
:10F7F60070726F6D203A20202E2E2E200D0A005397
:10F80600657074656D6272652000204846494E54E5
:10F816004F5343200044696D616E6368652000564E
:10F82600656E647265646920004D65726372656415
:10F83600692000446563656D62726520004E6F76CF
:10F84600656D6272652000204C46494E544F534305
:10F85600004F63746F62726520004A75696C6C654F
:10F866007420004665767269657220004A616E767C
:10F87600696572200053616D656469200065727266
:10F8860065757220004A6575646920004D61726471
:10F896006920004C756E646920004572726F722093
:10F8A60000417672696C2000416F757420004A75BC
:10F8B600696E20004D617273200020464F5343004D
:10F8C6004D6169200020200020416C61726D652029
:10F8D60076696120696E74657272757074696F6E8F
:10F8E600203A20736F7274696520414C4552544525
:10F8F60020494E41323236202D3E20524230206978
:10F906006E707574200D0A0020553B32343B30383A
:10F916003B31373B31383B33363B30342320207084
:10F926006F757220323420416F7574203230313752
:10F93600202031384833362030343D4A65756469B5
:10F946000D0A0D0A0020416C657274204D41534B1F
:10F956005F454E5F524547207265676973746572ED
:10F9660020303768203C2D2031302E30303020704A
:10F976006F7572203235306D410D0A000D0A205226
:10F98600617070656C20666F726D617420646520AD
:10F99600636465203A2022553B4A4A3B4D4D3B4124
:10F9A600413B48483B4D4D3B6A533B2322200D0AC1
:10F9B6000020436F6D70696C65206C65202573208F
:10F9C60061202573205554430D0A20617665632016
:10F9D60076657273696F6E20584338203A20202569
:10F9E60064200D0A0020415454454E54494F4E2080
:10F9F6003A20416472657373652049324320204C76
:10FA06004344203478323020646566696E69652027
:10FA160064616E73203A0D0A002052656C6563744A
:10FA2600757265202076616C657572206465204D5F
:10FA360041534B5F454E5F52454720726567697378
:10FA460074657220303768200D0A00204D61736B93
:10FA56002F416C65727420204D41534B5F454E5FBC
:10FA6600524547207265676973746572203036683F
:10FA7600203C2D203078383030310D0A0020436884
:10FA8600617267656D656E7420636172616374652A
:10FA96007265732053706563696175782073657448
:10FAA60020233120656E20434752414D0D0A002028
:10FAB60053617576652076616C6575722064616E3A
:10FAC6007320204D41534B5F454E5F524547207290
:10FAD6006567697374657220303768200D0A0020E7
:10FAE6000D0A53657175656E6365206427496E69F5
:10FAF60074204C43442034783230207669612049A2
:10FB060032433120504346383537340D0A002053EE
:10FB16006575696C20616C61726D6520636F7572C5
:10FB260072616E7420656E206D4120533D31303018
:10FB360020E0203831392020203A0D0A00204020CC
:10FB4600646563696D616C20232534752020736FAD
:10FB56006974204044657669636520376269747309
:10FB6600203D2030582530325820002043616C69F2
:10FB760062726174696F6E2072656769737465720B
:10FB860020303568203C2D20307830443142200D1D
:10FB96000A0020546573742070726573656E636520
:10FBA6002064657669636573207375722042757388
:10FBB60020493243310D0A002046696E20646520D3
:10FBC600706172616D65747261676520494E41327C
:10FBD60032362E2E2E204F4B0D0A0D0A0020766946
:10FBE60061206C69676E652023646566696E6520B1
:10FBF6004C43445F414444522030787878200D0AC3
:10FC060000204E455720536575696C206427616C4A
:10FC1600657274652025332E336620416D706572DA
:10FC260065730D0A0020436F6E6669672020494E92
:10FC3600413232365F434F4E465F5245472C30784D
:10FC460034313237200D0A000D0A4572726575721D
:10FC560020737572204A6F75722053656D61696EE7
:10FC660065206A532E200D0A0020426F75636C656D
:10FC7600207072696E636970616C65202070726FA6
:10FC86006772616D6D65200D0A002030783237206D
:10FC9600617665632050726F746F204261736520D0
:10FCA60031384632374B34320D0A002061647265B2
:10FCB600737365204C43443D20256420736F69743B
:10FCC60020305825303258200D0A002054657374B0
:10FCD6002042757A7A65722073757220736F72741A
:10FCE600696520524332200D0A00204D65737572F6
:10FCF6006520646520636F7572616E7420252035FA
:10FD060064206D41200D0A00204C43445F34626933
:10FD160074735F4932435F323032332D30383130BD
:10FD26002E680D0A00456570726F6D2032344C43A3
:10FD3600787878203235366B206F75203531324B26
:10FD46000020416666696368616765207375722085
:10FD56004C43442034783230200D0A0020494E416D
:10FD6600204D616E7566616374756572202030780A
:10FD7600253034580D0A0020494E41204964656EED
:10FD860074696669616E74203078253034580D0ABE
:10FD960000205043463837353420666F72204C4376
:10FDA6004420327831366361727300202520332E69
:10FDB600336620572020536575696C3D25322E33F6
:10FDC6006620410045637269747572652044533339
:10FDD6003233312E2E2E204F4B0D0A0020496E69EC
:10FDE600745F493243282920E0203130304B687A4D
:10FDF6003B0D0A00494E413232365F496E69745FE7
:10FE0600436F6E666967200D0A000D0A2048656C0F
:10FE16007020436F6D6D616E646573203A0D0A0044
:10FE260020496E6974204E434F3120E02031303036
:10FE360030487A0D0A002025332E326620562020BF
:10FE460025332E336620412020202000494E4132A2
:10FE560032362043757272656E742073656E736FE9
:10FE660072002056657273696F6E2050726F6772EA
:10FE7600616D6D652020002020494E4132323620CA
:10FE86005465737473203230323520003132333486
:10FE9600353637383930313233343536373839300C
:10FEA60000436172616374657265732053706563A4
:10FEB6006961757832004142434445464748494A9C
:10FEC6004B4C4D4E4F505152535400202025322E4C
:10FED60033662056202025322E336620412000200E
:10FEE6006D76413D25203564206D76553D252035BE
:10FEF600642000323032352D3032323420313846EB
:10FF060032374B3432005043463835373441203887
:10FF16006269747320492F4F00204E6220626F750C
:10FF2600636C65733D2535642020004C43442032C4
:10FF3600313139203278313663617273005043466D
:10FF46003835373420386269747320494F002050A1
:10FF5600726573656E746174696F6E203A00205520
:10FF66003D252035642020413D252035640045454A
:10FF760050524F4D20353132627974657300253504
:10FF860064204146463D25316420004F4C454420BF
:10FF960053534431333036006E6F6E20636F6E6E8E
:10FFA6007520210046656220323420323032350019
:10FFB6005254432044533332333100206B3D2025C5
:10FFC60035642020002048656C70200D0A00313011
:10FFD6003A35323A35340052656375203A00494E57
:10FFE60046004E414E00696E66006E616E006C6C96
:0AFFF6007300202E31006C6600003D
:020000040001F9
:10000000000E00017C6F000E7B6F62C08DF063C03C
:100010008EF064C08FF065C090F090BF14EF80F058
:1000200012EF80F02AEF80F0000E7C6F010E7B6FE4
:100030008DC003F08EC004F08FC005F090C006F0B4
:1000400055ECB5F003C08DF004C08EF005C08FF004
:1000500006C090F0000E0001946F000E936F68C10F
:100060007FF069C180F07B517C11D8A43AEF80F019
:100070003CEF80F043EF80F0EAA541EF80F043EFE2
:1000800080F05DEF80F07B517C11D8A44AEF80F0C6
:100090004CEF80F052EF80F0000E686F2B0E676F10
:1000A00056EF80F0000E686F2D0E676F67C008F284
:1000B000934B942B7F07D8A080078DC003F08EC090
:1000C00004F08FC005F090C006F016ECA8F0030411
:1000D0000410D8A46EEF80F070EF80F0BAEF80F0DB
:1000E000BF0E576EFF0E586E00016651596E5A6A68
:1000F0005750592658505A225A5007E11A0E595C47
:10010000D8B085EF80F087EF80F095EF80F0080E93
:100110009325076E020E9421086EE40E096EFF0E01
:100120000A6EAFECB1F0A1EF80F0080E9325076ED8
:10013000020E9421086EEC0E096EFF0E0A6EAFECF3
:10014000B1F00001FD0E7F27FF0E802360C013F089
:1001500061C014F0080E156E020E166E7FC017F007
:1001600080C018F0A7ECAAF013C060F014C061F0D2
:1001700006EF86F08DC003F08EC004F08FC005F04E
:1001800090C006F016ECA8F003500410D8A4CBEFF2
:1001900080F0CDEF80F000EF81F0BF0E576EFF0EC4
:1001A000586E00016651596E5A6A57505926585078
:1001B0005A225A5007E11A0E595CD8B0E2EF80F08B
:1001C000E4EF80F0F2EF80F0080E9325076E020E48
:1001D0009421086EE80E096EFF0E0A6EAFECB1F0C6
:1001E000A1EF80F0080E9325076E020E9421086E91
:1001F000F00E096EFF0E0A6EAFECB1F0A1EF80F0C9
:10020000000E0001956F000E966F800E976F3F0EE7
:10021000986F000E926F000E916F8DC003F08EC02C
:1002200004F08FC005F090C006F0000E076E000EBF
:10023000086E000E096E000E0A6E1BECACF0D8B012
:1002400024EF81F026EF81F0A9EF81F045EF81F0F6
:1002500095C011F096C012F097C013F098C014F03A
:10026000000E156E000E166E200E176E410E186EE3
:10027000E0EC93F011C095F012C096F013C097F027
:1002800014C098F00001914B922B8DC02AF08EC0C3
:100290002BF08FC02CF090C02DF0000E156E000ECC
:1002A000166E200E176E410E186E95C011F096C096
:1002B00012F097C013F098C014F0E0EC93F011C066
:1002C0002EF012C02FF013C030F014C031F013EC38
:1002D000A7F0D8B06EEF81F070EF81F028EF81F0D9
:1002E00090EF81F095C02AF096C02BF097C02CF0CB
:1002F00098C02DF0000E2E6E000E2F6E200E306E68
:10030000410E316E07EC96F02AC095F02BC096F0A6
:100310002CC097F02DC098F000019107D8A092074B
:100320008DC02AF08EC02BF08FC02CF090C02DF025
:1003300095C02EF096C02FF097C030F098C031F0E5
:1003400013ECA7F0D8A0A7EF81F0A9EF81F072EF2E
:1003500081F066C009F00A6A55ECB4F0095000015A
:10036000826F82C081F0670E8219D8A4BAEF81F043
:10037000BCEF81F0E2EF81F0E851E911D8A4C3EFBE
:1003800081F0C5EF81F0C9EF81F0000EE96F010E39
:10039000E86FE9BFD6EF81F0E95106E1E805D8B092
:1003A000D4EF81F0D6EF81F0DCEF81F0000E7E6FAC
:1003B000060E7D6FEBEF81F0E8C07DF0E9C07EF0C6
:1003C000EBEF81F0E9BFE7EF81F0E9EF81F0D6EFE5
:1003D00081F0DCEF81F0670E8219D8A4F2EF81F092
:1003E000F4EF81F023EF82F092AF02EF82F0FC0E87
:1003F000915DFF0E9259D8A000EF82F002EF82F0DB
:1004000021EF82F0FF0E576EFF0E586E7DC059F03F
:100410007EC05AF05750592658505A229151595C73
:100420005A50800A5B6E9251800A5B58D8A01BEF2D
:1004300082F01DEF82F021EF82F0660E816F23EFD4
:1004400082F0650E816F7DC073F07EC074F0670E20
:100450008219D8A42EEF82F030EF82F040EF82F0C4
:10046000660E8119D8A437EF82F039EF82F042EF9F
:1004700082F092BF40EF82F03EEF82F042EF82F0D6
:10048000734B742B660E8119D8A449EF82F04BEFA1
:1004900082F06BEF82F092BF52EF82F050EF82F069
:1004A0005EEF82F0000E956F000E966F800E976FD4
:1004B0003F0E986F000E926F000E916F670E8219BB
:1004C000D8B465EF82F067EF82F06BEF82F0915164
:1004D000732792517423000E8C6F000E8B6F8DC0AA
:1004E00083F08EC084F08FC085F090C086F095C0F8
:1004F00075F096C076F097C077F098C078F0FCEF72
:1005000082F083C02AF084C02BF085C02CF086C016
:100510002DF095C02EF096C02FF097C030F098C007
:1005200031F007EC96F02AC043F02BC044F02CC009
:1005300045F02DC046F09DEC9DF043C087F044C0CF
:1005400088F045C089F046C08AF087C003F088C0B3
:1005500004F089C005F08AC006F090ECA6F003C054
:1005600079F004C07AF083C02AF084C02BF085C0F3
:100570002CF086C02DF095C015F096C016F097C0EF
:1005800017F098C018F087C011F088C012F089C029
:1005900013F08AC014F0E0EC93F011C02EF012C0FA
:1005A0002FF013C030F014C031F078ECB4F02AC052
:1005B00083F02BC084F02CC085F02DC086F095C050
:1005C0002AF096C02BF097C02CF098C02DF0000EAA
:1005D0002E6E000E2F6E200E306E410E316E07EC27
:1005E00096F02AC095F02BC096F02CC097F02DC045
:1005F00098F000018B4B8C2B73518B5D8C51800AD2
:10060000576E7451800A5758D8A009EF83F00BEF4A
:1006100083F081EF82F095C011F096C012F097C080
:1006200013F098C014F0000E156E000E166EA00E9A
:10063000176E400E186EE0EC93F011C087F012C0F8
:1006400088F013C089F014C08AF083C02AF084C0F7
:100650002BF085C02CF086C02DF087C02EF088C00E
:100660002FF089C030F08AC031F013ECA7F0D8B079
:100670003CEF83F03EEF83F049EF83F0000E000182
:10068000876F000E886F000E896F000E8A6F72EF01
:1006900083F083C003F084C004F085C005F086C0F9
:1006A00006F087C007F088C008F089C009F08AC04A
:1006B0000AF01BECACF0D8A060EF83F062EF83F09F
:1006C00072EF83F0000179B168EF83F06AEF83F095
:1006D00072EF83F0000E876F000E886F000E896F37
:1006E000000E8A6F8DC003F08EC004F08FC005F03D
:1006F00090C006F087C007F088C008F089C009F0F4
:100700008AC00AF080EC91F003C083F004C084F04A
:1007100005C085F006C086F083C02AF084C02BF0A7
:1007200085C02CF086C02DF0000E156E000E166EE2
:10073000200E176E410E186E75C011F076C012F0C3
:1007400077C013F078C014F0E0EC93F011C02EF0F5
:1007500012C02FF013C030F014C031F013ECA7F02A
:10076000D8A0B5EF83F0B7EF83F0E0EF83F000019E
:10077000914B922B75C011F076C012F077C013F038
:1007800078C014F0000E156E000E166E200E176E57
:10079000410E186EE0EC93F011C075F012C076F0C7
:1007A00013C077F014C078F0660E00018119D8A448
:1007B000DCEF83F0DEEF83F0E0EF83F0734B742B1C
:1007C00075C095F076C096F077C097F078C098F035
:1007D000650E00018119D8B4F0EF83F0F2EF83F0D9
:1007E000F8EF83F091C071F092C072F0FCEF83F0EB
:1007F000000E726F000E716F000E706F000E6F6F43
:10080000000E6E6F000E6D6F000E8C6F000E8B6F02
:10081000F7EF84F083C02AF084C02BF085C02CF061
:1008200086C02DF095C02EF096C02FF097C030F006
:1008300098C031F007EC96F02AC043F02BC044F08A
:100840002CC045F02DC046F09DEC9DF043C087F0D4
:1008500044C088F045C089F046C08AF087C003F0E4
:1008600088C004F089C005F08AC006F090ECA6F0BC
:1008700003C079F004C07AF00001EAB942EF84F0D5
:1008800044EF84F061EF84F079517A11D8A44BEFF2
:1008900084F04DEF84F061EF84F0670E8219D8A4E4
:1008A00054EF84F056EF84F061EF84F072BF5DEF97
:1008B00084F05BEF84F061EF84F06D4B6E2BABEF57
:1008C00084F06F517011D8A468EF84F06AEF84F05F
:1008D00094EF84F072BF71EF84F06FEF84F094EFC7
:1008E00084F0080E9325D96E020E9421DA6E2E0E36
:1008F000DF6E934B942B7F07D8A08007000E706F9C
:10090000010E6F6F94EF84F0080E9325D96E020EDE
:100910009421DA6E300EDF6E934B942B7F07D8A0B4
:1009200080076D07D8A06E076D516E11D8A49BEF9C
:1009300084F09DEF84F084EF84F0080E9325D96E47
:10094000020E9421DA6E7951300FDF6E934B942BA7
:100950007F07D8A0800783C02AF084C02BF085C011
:100960002CF086C02DF095C015F096C016F097C0FB
:1009700017F098C018F087C011F088C012F089C035
:1009800013F08AC014F0E0EC93F011C02EF012C006
:100990002FF013C030F014C031F078ECB4F02AC05E
:1009A00083F02BC084F02CC085F02DC086F095C05C
:1009B0002AF096C02BF097C02CF098C02DF0000EB6
:1009C0002E6E000E2F6E200E306E410E316E07EC33
:1009D00096F02AC095F02BC096F02CC097F02DC051
:1009E00098F000017107D8A072078B4B8C2B7351C4
:1009F0008B5D8C51800A576E7451800A5758D8B05D
:100A000004EF85F006EF85F014EF85F094BF12EF48
:100A100085F0945109E14B0E935DD8A012EF85F05B
:100A200014EF85F00AEF84F06F517011D8A41BEF1A
:100A300085F01DEF85F02EEF85F0EAA922EF85F015
:100A400024EF85F02EEF85F0080E9325D96E020E67
:100A50009421DA6E2E0EDF6E934B942B080E9325A5
:100A6000D96E020E9421DA6E000EDF6E650E8119CA
:100A7000D8A43DEF85F03FEF85F0A6EF80F0000EA3
:100A80008C6F4F0E8B6F080E8B25D96E020E8C214A
:100A9000DA6E000EDF6E000E7C6F000E7B6F92BF71
:100AA00056EF85F054EF85F05EEF85F0000E7C6F19
:100AB000010E7B6F916D921FD8B0922B000E7E6F4E
:100AC000020E7D6F8FEF85F08B07D8A08C07080E84
:100AD0008B25D96E020E8C21DA6E91C003F092C084
:100AE00004F0000E066E0A0E056E6CECABF00350BF
:100AF000300FDF6E91C003F092C004F0000E066E5E
:100B00000A0E056E0AECABF003C091F004C092F03F
:100B100000017D07D8A07E077F07D8A080079151EC
:100B20009211D8A496EF85F098EF85F064EF85F0E8
:100B30007EBFA5EF85F07E5106E17D05D8B0A3EF1D
:100B400085F0A5EF85F064EF85F08B07D8A08C07C2
:100B50007B517C11D8A4AFEF85F0B1EF85F0B7EFF2
:100B600085F0000E6A6F2B0E696FBBEF85F0000EEB
:100B70006A6F2D0E696F080E8B25D96E020E8C21BF
:100B8000DA6E6000A7F1DFFF7F07D8A080078B0730
:100B9000D8A08C07BF0E576EFF0E586E6651596E67
:100BA0005A6A5750592658505A225A5009E11A0E7B
:100BB000595CD8A0DEEF85F0E0EF85F0E6EF85F038
:100BC000000E6C6F650E6B6FEAEF85F0000E6C6FB8
:100BD000450E6B6F080E8B25D96E020E8C21DA6ED6
:100BE0006000AFF1DFFF7F07D8A08007080E9325D4
:100BF000076E020E9421086E080E8B25096E020EF8
:100C00008C210A6EAFECB1F0A6EF80F01200600EFE
:100C10003901D96F000EDB6F000EDD6F080EDF6F3C
:100C2000000EDE6F090E0101FC6F1E0EFB6FE40E5D
:100C3000E82EFED7FB2FFCD7FC2FFAD700F0D29E70
:100C40003901909F000E3A01456F000E466F000E6D
:100C5000476F000E656F000E666F000E676F3901FB
:100C6000909F9191A09FA191E1ECA9F0000E00014D
:100C7000F56F000EF46F000EF425D96E040EF52109
:100C8000DA6E000EDF6EF44BF52BF55109E1800EA4
:100C9000F45DD8A04EEF86F050EF86F03BEF86F083
:100CA000000EF56F000EF46F200EF425D96E030EC2
:100CB000F521DA6E000EDF6EF44BF52BF55109E1EC
:100CC000800EF45DD8A067EF86F069EF86F054EFF0
:100CD00086F0000EF56F000EF46F580EF425D96EF5
:100CE000020EF521DA6E000EDF6EF44BF52BF55196
:100CF00009E14F0EF45DD8A080EF86F082EF86F018
:100D00006DEF86F0000EF06F040EF16F0EECB4F094
:100D1000090E0101FC6F1E0EFB6FE40EE82EFED7DC
:100D2000FB2FFCD7FC2FFAD700F024ECB6F0540EC2
:100D3000036EFF0E046EC9ECB2F024ECB6F0000EA8
:100D40000001F56F000EF46FD890F435D96EF535CB
:100D5000DA6EC20ED926020EDA226F0078FF03F097
:100D60006F0074FF04F0C9ECB2F0BA78090E01010B
:100D7000FC6F1E0EFB6FE40EE82EFED7FB2FFCD798
:100D8000FC2FFAD700F00001F44BF52BF55109E1E7
:100D9000090EF45DD8A0CFEF86F0D1EF86F0A4EF76
:100DA00086F024ECB6F024ECB6F0F0C0C9F0F1C047
:100DB000CAF0B70E0001CB6FF90ECC6FAA0ECD6F43
:100DC000FF0ECE6FD40ECF6FFF0ED06F090ED26F15
:100DD000380ED16F1EECB3F0F0C003F0F1C004F098
:100DE00040ECB1F024ECB6F0260E036EFE0E046E5D
:100DF000C9ECB2F0A4ECAFF0D10E036EFC0E046EA1
:100E0000C9ECB2F0090E0101FC6F1E0EFB6FE40E7F
:100E1000E82EFED7FB2FFCD7FC2FFAD700F03F01BE
:100E20003E9FC484090E0101FC6F1E0EFB6FE40E91
:100E3000E82EFED7FB2FFCD7FC2FFAD700F0C49486
:100E40003F013E8F110E0101FC6F3C0EFB6FCB0E7C
:100E5000E82EFED7FB2FFCD7FC2FFAD73F013E9F91
:100E6000C48424ECB6F0E20E036EFD0E046EC9ECF1
:100E7000B2F0F9ECB6F0980E036EFB0E046EC9ECFE
:100E8000B2F056EC9CF024ECB6F0270E0001FB6F9C
:100E9000EB0E036EF90E046EC9ECB2F00E0E036E8B
:100EA000FD0E046EC9ECB2F0E30E036EFB0E046E91
:100EB000C9ECB2F0900E036EFC0E046EC9ECB2F0F9
:100EC00024ECB6F0000E5D6E140E5C6E270E000171
:100ED000FB6F580EC96F020ECA6FB10ECB6FFC0EBE
:100EE000CC6FFBC0CDF0CE6BFBC0CFF0D06B1EEC57
:100EF000B3F0580E036E020E046E40ECB1F0E50E36
:100F0000036EFA0E046EC9ECB2F0D3ECA4F024EC3C
:100F1000B6F0010EDEECAEF0090E0101FC6F1E0E04
:100F2000FB6FE40EE82EFED7FB2FFCD7FC2FFAD781
:100F300000F0020EDEECAEF0090E0101FC6F1E0E99
:100F4000FB6FE40EE82EFED7FB2FFCD7FC2FFAD761
:100F500000F0470E036EFD0E046EC9ECB2F0BC0E3D
:100F6000216EFE0E226E1EECB0F0000E276E020EF9
:100F7000266E44ECAAF0920E216EFE0E226E1EEC3E
:100F8000B0F0000E276E030E266E44ECAAF0680E39
:100F9000216EFE0E226E1EECB0F0000E276E040EC7
:100FA000266E44ECAAF0F90E216EFE0E226E1EECA7
:100FB000B0F0020EF4ECB2F0000E0001F56F000E7E
:100FC000F46F830E036EFA0E046EC9ECB2F0010EDC
:100FD000DEECAEF0D00E0101FB6FC90EE82EFED79D
:100FE000FB2FFCD700D0000E276E010E266E44ECBE
:100FF000AAF0A70E216EFE0E226E1EECB0F0000EBF
:10100000276E020E266E44ECAAF0D00E0101FB6F93
:10101000C90EE82EFED7FB2FFCD700D0000E236EA2
:10102000000E226E34ECA4F024ECB6F0000E0101A8
:10103000776F000E766F000E756F000E746FFA0EEC
:10104000036EFD0E046EC9ECB2F0D4EC97F06F0E97
:10105000036EFC0E046EC9ECB2F0CE0E036EF80EF9
:10106000046EC9ECB2F070ECB2F03901A19191813B
:10107000D28EC494400E0001FB6F000E0101C16FBF
:10108000000EC26FC10E0001EC6F010EED6F020E7B
:10109000186EECC019F0EDC01AF0000E1C6E030EB5
:1010A0001B6EFB5122ECAFF00101C151FC6FFB6BD9
:1010B000C251FB25746F000EFC21756F400E0001BC
:1010C000FB6F000E0101C16F000EC26FC10E000167
:1010D000EC6F010EED6F010E186EECC019F0EDC053
:1010E0001AF0000E1C6E030E1B6EFB5122ECAFF0CB
:1010F0000101C151FC6FFB6BC251FB25766F000EE5
:10110000FC21776F400E0001FB6F000E0101C16FE3
:10111000000EC26FC10E0001EC6F010EED6F060EE6
:10112000186EECC019F0EDC01AF0000E1C6E020E25
:101130001B6EFB5122ECAFF00101C151FC6FFB6B48
:10114000C251FB25726F000EFC21736F72C1FBF15F
:1011500073C1FCF1040EFD6FD890FC33FB33FD2FFF
:10116000ACEF88F0FB510F0BB86F400E0001FB6F26
:10117000000E0101C16F000EC26FC10E0001EC6FC5
:10118000010EED6F030E186EECC019F0EDC01AF0F1
:10119000000E1C6E030E1B6EFB5122ECAFF0010122
:1011A000C151FC6FFB6BC251FB250001FD6F0101BA
:1011B000000EFC210001FE6FFDC003F0FEC004F034
:1011C000056A066A000EA8EC9FF003C02AF004C06E
:1011D0002BF005C02CF006C02DF0000E2E6E400E38
:1011E0002F6E1C0E306E450E316E07EC96F02AC045
:1011F00052F12BC053F12CC054F12DC055F1010117
:10120000B805D8A406EF89F008EF89F009EF89F056
:10121000BA98000E0001F06F040EF16FF0C0C9F033
:10122000F1C0CAF0840ECB6FFF0ECC6F9AC1CDF027
:101230009BC1CEF0B8C1CFF0D06B1EECB3F0000E66
:101240000201586F580E0001C96F020ECA6FE50EF9
:10125000CB6FFE0ECC6F76C1CDF077C1CEF074C1EE
:10126000CFF075C1D0F01EECB3F0F0C011F0F1C0BA
:1012700012F0580E136E020E146EE6ECB6F0AE0EBF
:10128000156E470E166EA10E176E3F0E186E74C1C6
:1012900003F075C104F0056A066A000EA8EC9FF021
:1012A00003C011F004C012F005C013F006C014F022
:1012B000E0EC93F011C02AF012C02BF013C02CF018
:1012C00014C02DF0000E2E6E000E2F6E7A0E306EB2
:1012D000440E316E07EC96F02AC04AF12BC04BF158
:1012E0002CC04CF12DC04DF1000E156E000E166E87
:1012F000200E176E400E186E76C103F077C104F011
:10130000000E04BEFF0E056E066E010EA8EC9FF0E7
:1013100003C011F004C012F005C013F006C014F0B1
:10132000E0EC93F011C02AF012C02BF013C02CF0A7
:1013300014C02DF0000E2E6E500E2F6EC30E306EA8
:10134000470E316E07EC96F02AC04EF12BC04FF1DC
:101350002CC050F12DC051F1580E0001C96F020E82
:10136000CA6FD10ECB6FFE0ECC6F4AC1CDF04BC110
:10137000CEF04CC1CFF04DC1D0F04EC1D1F04FC135
:10138000D2F050C1D3F051C1D4F01EECB3F0F0C094
:1013900011F0F1C012F0580E136E020E146EE6EC4E
:1013A000B6F0580E0001C96F020ECA6FB10ECB6FB6
:1013B000FD0ECC6F52C1CDF053C1CEF054C1CFF071
:1013C00055C1D0F046C1D1F047C1D2F048C1D3F0E9
:1013D00049C1D4F01EECB3F0F0C011F0F1C012F02E
:1013E000580E136E020E146EE6ECB6F0F0C003F069
:1013F000F1C004F040ECB1F024ECB6F0270E00018F
:10140000FB6F04ECA6F03F013E9FC484BA88E2EC77
:10141000AFF07A0E0101FC6FC10EFB6F810EE82E5A
:10142000FED7FB2FFCD7FC2FFAD700D00101C00557
:10143000D8A41DEF8AF01FEF8AF0D9EF8BF0DD0EF4
:10144000036EFF0E046EC9ECB2F0200E0001EE6FC9
:10145000030EEF6FEEC003F0EFC004F040ECB1F00C
:1014600024ECB6F06000BBF3D9FF6000BFF3DAFFF5
:10147000480EDE18D8A43FEF8AF041EF8AF08EEFD5
:101480008AF0000120EE01F0EE51D926EF51DA2268
:10149000650EDE18D8A44FEF8AF051EF8AF08EEF78
:1014A0008AF020EE02F0EE51D926EF51DA226C0ECE
:1014B000DE18D8A45EEF8AF060EF8AF08EEF8AF033
:1014C00020EE03F0EE51D926EF51DA22700EDE182D
:1014D000D8A46DEF8AF06FEF8AF08EEF8AF0100ECD
:1014E000036EFE0E046EC9ECB2F0140E036EFB0E1A
:1014F000046EC9ECB2F0CB0E036EFF0E046EC9ECA5
:10150000B2F0200E036E030E046E40ECB1F024EC3A
:10151000B6F0000E0001EE6F000EEF6F6000BBF33F
:10152000D9FF6000BFF3DAFF530EDE18D8A49BEF9B
:101530008AF09DEF8AF0D9EF8BF0000120EE01F0E8
:10154000EE51D926EF51DA223D0EDE18D8A4ABEFCA
:101550008AF0ADEF8AF0D9EF8BF0EEC003F0EFC068
:1015600004F09DECB2F0050E03180410D8A4BBEFF4
:101570008AF0BDEF8AF0D9EF8BF0000120EE02F087
:10158000EE51D926EF51DA22DF50D00FFC6FFC511B
:10159000640D6F00CCFFFDF06F00D0FFFEF020EE79
:1015A00003F0EE51D926EF51DA22DF50D00FFC6F55
:1015B000FC510A0D6F00CCFFFBF16F00D0FFFCF176
:1015C000FD510101FB250001FD6FFE510101FC21D0
:1015D0000001FE6F20EE04F0EE51D926EF51DA2221
:1015E000DF50D00FFC6FFC51FD25FD6F000EFE217A
:1015F000FE6FFE5109E1640EFD5DD8A002EF8BF095
:1016000004EF8BF0D4EF8BF0340EFD5D030EFE592A
:10161000D8B00DEF8BF00FEF8BF0D4EF8BF0FDC057
:1016200003F0FEC004F0000E066E280E056E95EC69
:10163000B6F003C0FDF004C0FEF0580E0001C96F03
:10164000020ECA6FC10ECB6FFF0ECC6FFDC0CDF086
:10165000FEC0CEF01EECB3F0580E036E020E046E08
:1016600040ECB1F039019191B50E036EFA0E046EA3
:10167000C9ECB2F0070E0101C16F0001FE5101017A
:10168000C26FFDC0C3F1400E0001FB6FC10EEC6FD5
:10169000010EED6F030EFC6FECC018F0EDC019F0F9
:1016A000FCC01AF01B6AFB5113ECB2F01F0E036E64
:1016B000FA0E046EC9ECB2F0400E0001FB6F000E92
:1016C0000101C16F000EC26FC10E0001EC6F010E6F
:1016D000ED6F070E186EECC019F0EDC01AF0000E99
:1016E0001C6E030E1B6EFB5122ECAFF00101C151C9
:1016F000FC6FFB6BC251FB250001FD6F0101000E69
:10170000FC210001FE6F170E156EB70E166E510EFE
:10171000176E3F0E186EFDC003F0FEC004F0056AA0
:10172000066A000EA8EC9FF003C011F004C012F08E
:1017300005C013F006C014F0E0EC93F011C02AF0DD
:1017400012C02BF013C02CF014C02DF0000E2E6E22
:10175000000E2F6E000E306E470E316E07EC96F0C5
:101760002AC046F12BC047F12CC048F12DC049F1E9
:10177000580E0001C96F020ECA6F070ECB6FFC0E28
:10178000CC6F46C1CDF047C1CEF048C1CFF049C1C2
:10179000D0F01EECB3F0580E036E020E046E40EC57
:1017A000B1F03901A1919181000E0001EE6F000EA0
:1017B000EF6F01019A4B9B2B39EF88F057EF00F048
:1017C00060006FF2D9FF600073F2DAFF6F007BFFF9
:1017D000F6FF6F0077FFF7FF000EF86E0800F55078
:1017E000250AD8A4F6EF8BF0F8EF8BF05CEF91F0C0
:1017F00060006FF2D9FF600073F2DAFFDE2A000E9C
:10180000DD22000E0101696F000E686F68C1EAF009
:1018100069C1EBF00001E869E969000EAE6F000EE6
:10182000AD6F61EF8CF0EA8160006FF2D9FF60006C
:1018300073F2DAFFDE2A000EDD2261EF8CF0EA831C
:1018400014EF8CF0EA8514EF8CF0EA8714EF8CF03B
:10185000EA8914EF8CF0000EAE6F010EAD6F61EFF0
:101860008CF060006FF2D9FF600073F2DAFF6F0056
:101870007BFFF6FF6F0077FFF7FF000EF86E0800A2
:10188000F5509F6FA06BA051000AD8B44AEF8CF0BE
:101890002BEF8CF09F51200AD8B425EF8CF0030A6F
:1018A000D8B428EF8CF0080AD8B422EF8CF0060ADE
:1018B000D8B413EF8CF01D0AD8B41FEF8CF02BEFC7
:1018C0008CF0AD51AE11D8B468EF8CF06AEF8CF0AB
:1018D00031EF8CF0EAA16FEF8CF071EF8CF072EFCA
:1018E0008CF0EA9360006FF2D9FF600073F2DAFFC8
:1018F0006F007BFFF6FF6F0077FFF7FF000EF86EBB
:101900000800F5502A0AD8A488EF8CF08AEF8CF0F2
:10191000C0EF8CF060006FF2D9FF600073F2DAFF65
:10192000DE2A000EDD22600077F2D9FF60007BF234
:10193000DAFF6F007CFF9FF0020EDE266F007CFF57
:10194000A0F0000EDD2260007FF2D9FF600083F27C
:10195000DAFF6F0078FF68F16F0074FF69F1010131
:1019600069BFB7EF8CF0B5EF8CF003EF8DF000019D
:10197000EA810101686D691FD8B0692B03EF8DF012
:1019800060006FF2D9FF600073F2DAFF6F0078FF3A
:101990000AF06F0074FF0BF01AECA2F00AC068F1B5
:1019A0000BC069F1DDEF8CF060006FF2D9FF6000D1
:1019B00073F2DAFFDE2A000EDD22D00E00019F6FE7
:1019C000FF0EA06F60006FF2D9FF600073F2DAFFC4
:1019D0006F007BFFF6FF6F0077FFF7FF000EF86EDA
:1019E0000800F550A16FA26B9F51A127A051A2231F
:1019F000A25109E10A0EA15DD8A001EF8DF003EF1D
:101A00008DF0D4EF8CF060006FF2D9FF600073F2BC
:101A1000DAFF6F007BFFF6FF6F0077FFF7FF000E26
:101A2000F86E0800F5502E0AD8A419EF8DF01BEFC0
:101A30008DF0ABEF8DF0000E0001E96F000EE86F46
:101A400060006FF2D9FF600073F2DAFFDE2A000E49
:101A5000DD2260006FF2D9FF600073F2DAFF6F00E1
:101A60007BFFF6FF6F0077FFF7FF000EF86E0800B0
:101A7000F5502A0AD8A43FEF8DF041EF8DF068EFC2
:101A80008DF060006FF2D9FF600073F2DAFFDE2A9A
:101A9000000EDD22600077F2D9FF60007BF2DAFFF2
:101AA0006F007CFF9FF0020EDE266F007CFFA0F02F
:101AB000000EDD2260007FF2D9FF600083F2DAFFC2
:101AC0006F0078FFE8F06F0074FFE9F0ABEF8DF086
:101AD00060006FF2D9FF600073F2DAFF6F0078FFE9
:101AE0000AF06F0074FF0BF01AECA2F00AC0E8F0E5
:101AF0000BC0E9F085EF8DF060006FF2D9FF600058
:101B000073F2DAFFDE2A000EDD22D00E00019F6F95
:101B1000FF0EA06F60006FF2D9FF600073F2DAFF72
:101B20006F007BFFF6FF6F0077FFF7FF000EF86E88
:101B30000800F550A16FA26B9F51A127A051A223CD
:101B4000A25109E10A0EA15DD8A0A9EF8DF0ABEF7B
:101B50008DF07CEF8DF060006FF2D9FF600073F2C2
:101B6000DAFF6F007BFFF6FF6F0077FFF7FF000ED5
:101B7000F86E0800F550096E0A6A55ECB4F0095089
:101B80000001B96FB951D8B4C8EF8DF0CAEF8DF02C
:101B900014EF8EF060006FF2D9FF600073F2DAFF8D
:101BA0006F0078FF9FF06F0074FFA0F0010E9F2779
:101BB000000EA02360007FF2F6FF600083F2F7FFC3
:101BC000000EF86E0800F550096E0A6A55ECB4F084
:101BD00009500001BA6FBA51D8B4F1EF8DF0F3EFAC
:101BE0008DF014EF8EF060006FF2D9FF600073F299
:101BF000DAFF6F0078FF9FF06F0074FFA0F0020E15
:101C00009F27000EA02360007FF2F6FF600083F2A2
:101C1000F7FF000EF86E0800F550096E0A6A55ECE1
:101C2000B4F009500001BB6F60006FF2D9FF600093
:101C300073F2DAFF6F007BFFF6FF6F0077FFF7FFAD
:101C4000000EF86E0800F550640AD8B42AEF8EF042
:101C50002CEF8EF044EF8EF060006FF2D9FF600041
:101C600073F2DAFF6F007BFFF6FF6F0077FFF7FF7D
:101C7000000EF86E0800F550690AD8A442EF8EF005
:101C800044EF8EF08EEF8EF060006FF2D9FF6000AF
:101C900073F2DAFFDE2A000EDD22600077F2D9FF50
:101CA00060007BF2DAFF6F007CFF9FF0020EDE2601
:101CB0006F007CFFA0F0000EDD2260007FF2D9FFF4
:101CC000600083F2DAFF6F0078FFA3F06F0074FF0B
:101CD000A4F0000EA4BFFF0EA56FA66FA76FA86F9C
:101CE000A96FAA6F99C01EF09AC01FF0A3C020F080
:101CF000A4C021F0A5C022F0A6C023F0A7C024F004
:101D0000A8C025F0A9C026F0AAC027F08EEC99F053
:101D10001EC099F01FC09AF07FEF91F0660EB919BE
:101D2000D8A495EF8EF097EF8EF0EAEF8EF060007A
:101D30006FF2D9FF600073F2DAFF6F007BFFF6FFEE
:101D40006F0077FFF7FF000EF86E08006F00D4FFFA
:101D5000C0F060006FF2D9FF600073F2DAFFDE2A94
:101D6000000EDD22600077F2D9FF60007BF2DAFF1F
:101D70006F007CFF9FF0040EDE266F007CFFA0F05A
:101D8000000EDD2260007FF2D9FF600083F2DAFFEF
:101D90006F0078FFBCF06F0078FFBDF06F0078FF38
:101DA000BEF06F0078FFBFF099C060F09AC061F09C
:101DB000BCC062F0BDC063F0BEC064F0BFC065F0DF
:101DC000C0C066F000EC80F060C099F061C09AF08D
:101DD0007FEF91F0B90E036E000E046EFC0E056EDF
:101DE000FF0E066E000E086E020E076E8BECA3F05F
:101DF00003500410D8A4FFEF8EF001EF8FF095EFA1
:101E00008FF060006FF2D9FF600073F2DAFF6F00AD
:101E100078FF9FF06F0074FFA0F0010E00019F2774
:101E2000000EA02360007FF2F6FF600083F2F7FF50
:101E3000000EF86E08006F00D4FFC0F0BF0E9F6F59
:101E4000FF0EA06F60006FF2D9FF600073F2DAFF3F
:101E50006F007BFFF6FF6F0077FFF7FF000EF86E55
:101E60000800F550A16FA26B9F51A127A051A2239A
:101E7000A25107E11A0EA15DD8B041EF8FF043EFF8
:101E80008FF067EF8FF0600077F2D9FF60007BF290
:101E9000DAFF6F007CFF9FF0040EDE266F007CFFF0
:101EA000A0F0000EDD2260007FF2D9FF600083F217
:101EB000DAFF6F0078FFBCF06F0078FFBDF06F00B5
:101EC00078FFBEF06F0078FFBFF089EF8FF0600001
:101ED00077F2D9FF60007BF2DAFF6F007CFF9FF0A2
:101EE000040EDE266F007CFFA0F0000EDD226000F5
:101EF0007FF2D9FF600083F2DAFF6F0078FFBCF059
:101F00006F0078FFBDF06F0078FFBEF06F0078FFC4
:101F1000BFF0020E60006FF2D9FF600073F2DAFFCB
:101F2000DE26000EDD22D4EF8EF060006FF2D9FFC6
:101F3000600073F2DAFF6F007BFFF6FF6F0077FF40
:101F4000F7FF000EF86E0800F550730AD8B4ABEF37
:101F50008FF0ADEF8FF0CCEF8FF060006FF2D9FF14
:101F6000600073F2DAFF6F0078FF03F06F0074FF18
:101F700004F0F40E056EFF0E066E000E086E030EE2
:101F8000076E8BECA3F003500410D8A4CAEF8FF0B7
:101F9000CCEF8FF026EF90F060006FF2D9FF600079
:101FA00073F2DAFF6F007BFFF6FF6F0077FFF7FF3A
:101FB000000EF86E0800F550730AD8B4E2EF8FF007
:101FC000E4EF8FF0EBEF8FF0000E0001B06F030E27
:101FD000AF6FF0EF8FF0000E0001B06F010EAF6F2A
:101FE00060006FF2D9FF600073F2DAFFAF51DE26B6
:101FF000B051DD22600077F2D9FF60007BF2DAFF9A
:102000006F007CFF9FF0020EDE266F007CFFA0F0C9
:10201000000EDD2260007FF2D9FF600083F2DAFF5C
:102020006F0078FFABF06F0074FFACF099C00CF05C
:102030009AC00DF0ABC00EF0ACC00FF082ECA0F077
:102040000CC099F00DC09AF07FEF91F060006FF234
:10205000D9FF600073F2DAFF6F007BFFF6FF6F00BD
:1020600077FFF7FF000EF86E0800F550750AD8A448
:102070003CEF90F03EEF90F08AEF90F060006FF24E
:10208000D9FF600073F2DAFFDE2A000EDD22600065
:1020900077F2D9FF60007BF2DAFF6F007CFF9FF0E0
:1020A000020EDE266F007CFFA0F0000EDD22600035
:1020B0007FF2D9FF600083F2DAFF6F0078FFA1F0B2
:1020C0006F0074FFA2F0A1C0B1F0A2C0B2F0000195
:1020D000B36BB46BB56BB66BB76BB86B99C01EF0D6
:1020E0009AC01FF0B1C020F0B2C021F0B3C022F0FE
:1020F000B4C023F0B5C024F0B6C025F0B7C026F0B8
:10210000B8C027F0A6EC9EF01EC099F01FC09AF050
:102110007FEF91F060006FF2D9FF600073F2DAFF99
:102120006F007BFFF6FF6F0077FFF7FF000EF86E82
:102130000800F550780AD8B4A0EF90F0A2EF90F024
:10214000BAEF90F060006FF2D9FF600073F2DAFF2F
:102150006F007BFFF6FF6F0077FFF7FF000EF86E52
:102160000800F550580AD8A4B8EF90F0BAEF90F0F4
:102170001AEF91F060006FF2D9FF600073F2DAFF9E
:102180006F007BFFF6FF6F0077FFF7FF000EF86E22
:1021900008006F00D4FFC0F060006FF2D9FF60004C
:1021A00073F2DAFFDE2A000EDD22600077F2D9FF3B
:1021B00060007BF2DAFF6F007CFF9FF0020EDE26EC
:1021C0006F007CFFA0F0000EDD2260007FF2D9FFDF
:1021D000600083F2DAFF6F0078FFA1F06F0074FFF8
:1021E000A2F0A1C0B1F0A2C0B2F00001B36BB46B19
:1021F000B56BB66BB76BB86B99C01EF09AC01FF089
:10220000B1C020F0B2C021F0B3C022F0B4C023F0BE
:10221000B5C024F0B6C025F0B7C026F0B8C027F08E
:10222000C0C028F001EC9BF01EC099F01FC09AF0CE
:102230007FEF91F060006FF2D9FF600073F2DAFF78
:102240006F007BFFF6FF6F0077FFF7FF000EF86E61
:102250000800F550250AD8A430EF91F032EF91F044
:102260004CEF91F060006FF2D9FF600073F2DAFF7B
:10227000DE2A000EDD22000E046E250E036E99C0CC
:1022800005F09AC006F00DECA9F0000E00019A6F5F
:10229000010E996F7FEF91F060006FF2D9FF60003F
:1022A00073F2DAFFDE2A000EDD22000E00019A6FC3
:1022B000000E996F7FEF91F060006FF2D9FF600020
:1022C00073F2DAFF6F007BFFF6FF6F0077FFF7FF17
:1022D000000EF86E0800F550036E046A99C005F010
:1022E0009AC006F00DECA9F060006FF2D9FF600013
:1022F00073F2DAFFDE2A000EDD2245EF91F01200C4
:102300000650800B0F6E06500624116E05AE8BEF43
:1023100091F08DEF91F08EEF91F011801150D8B4C3
:1023200094EF91F096EF91F0ABEF91F01128D8A4D3
:102330009CEF91F09EEF91F0A6EF91F0000E036EEE
:10234000000E046E000E056E000E066E058E000E69
:10235000066EB3EF91F0000E036E000E046E000ED9
:10236000056E000E066E0A50800B106E0F5010188E
:10237000D8B4BDEF91F0BFEF91F0C0EF91F00F8CAA
:102380000A500A24106E09AEC8EF91F0CAEF91F01E
:10239000CBEF91F010801050D8B4D1EF91F0D3EF83
:1023A00091F0E8EF91F01028D8A4D9EF91F0DBEF8D
:1023B00091F0E3EF91F0000E076E000E086E000E34
:1023C000096E000E0A6E098E000E0A6EF0EF91F093
:1023D000000E076E000E086E000E096E000E0A6EEB
:1023E0001150105CD8B0F7EF91F0F9EF91F020EFB9
:1023F00092F00FACFEEF91F000EF92F002EF92F04E
:10240000800E0F1A11C012F010C011F012C010F09F
:1024100003C012F007C003F012C007F004C012F0AE
:1024200008C004F012C008F005C012F009C005F0A1
:1024300012C009F006C012F00AC006F012C00AF07D
:10244000000E126E115010C00BF00C6A0B5E000EE5
:102450000C5A0CBE35EF92F00C5009E11A0E0B5CD1
:10246000D8A035EF92F037EF92F06EEF92F0035074
:10247000041005100610D8A440EF92F043EF92F03C
:10248000010E44EF92F0000E126E000E036E000E6D
:10249000046E000E056E000E066E10C011F077EF90
:1024A00092F012A056EF92F058EF92F05EEF92F099
:1024B000D89012300109126E60EF92F0D89012326B
:1024C00003A065EF92F067EF92F068EF92F0128E42
:1024D00006340632053204320332112A1050115CE0
:1024E000D8A075EF92F077EF92F051EF92F00FBC19
:1024F0007CEF92F07EEF92F0BEEF92F01150D8A4F4
:1025000084EF92F086EF92F090EF92F0000E036E5F
:10251000000E046E000E056E000E066EDFEF93F0E7
:102520000750032608500422095005220A500622AB
:1025300006A09DEF92F09FEF92F04BEF93F012A068
:10254000A4EF92F0A6EF92F0ACEF92F0D890123098
:102550000109126EAEEF92F0D890123203A0B3EFE1
:1025600092F0B5EF92F0B6EF92F0128E063406328A
:10257000053204320332112A4BEF93F00750035C0B
:1025800008500458095005580650800A0B6E0A502E
:10259000800A0B58D8B0CFEF92F0D1EF92F0FCEF59
:1025A00092F00350075C0B6E045008580C6E0550F7
:1025B00009580D6E06500A580E6EFF0E0B24036E5E
:1025C000FF0E0C20046EFF0E0D20056EFF0E0E2078
:1025D000066E800E0F1A126C1250D8A4F2EF92F011
:1025E000F4EF92F004EF93F0010E0326000E0422A4
:1025F0000522062204EF93F00750035E0850045AA8
:102600000950055A0A50065A0350041005100610C6
:10261000D8A40DEF93F00FEF93F044EF93F0125026
:10262000D8A415EF93F017EF93F044EF93F0000E5A
:10263000036E000E046E000E056E000E066EDFEFD8
:1026400093F0D890033604360536063612AE2BEFDB
:1026500093F02DEF93F02EEF93F0038012A033EF61
:1026600093F035EF93F039EF93F0D88012363BEFCB
:1026700093F0D89012361150D8B441EF93F043EF55
:1026800093F044EF93F0110605AE49EF93F04BEF52
:1026900093F021EF93F0000E106E12AE52EF93F014
:1026A00054EF93F06CEF93F012C00BF07F0E0B160B
:1026B000D8B45DEF93F05FEF93F063EF93F0010E0A
:1026C000106E6CEF93F003A068EF93F06AEF93F055
:1026D0006CEF93F05FEF93F01050D8B472EF93F07B
:1026E00074EF93F09FEF93F0010E0326000E042287
:1026F0000522062206A07FEF93F081EF93F09FEF73
:1027000093F003C00BF004C00CF005C00DF006C040
:102710000EF00E340E320D320C320B320BC003F0C1
:102720000CC004F00DC005F00EC006F01128D8B49E
:102730009CEF93F09EEF93F09FEF93F0112A1128F6
:10274000D8B4A5EF93F0A7EF93F0AFEF93F011504B
:10275000D8A4ADEF93F0AFEF93F0C1EF93F0000E7C
:10276000036E000E046E000E056E000E066E115014
:10277000D8A4BDEF93F0BFEF93F0C1EF93F0000E3C
:102780000F6E11A0C6EF93F0C8EF93F0CBEF93F06C
:10279000058ECCEF93F0059ED8901130066E0FAEEB
:1027A000D4EF93F0D6EF93F0D7EF93F0068E03C0FB
:1027B00003F004C004F005C005F006C006F01200E6
:1027C0001450800B1D6E14501424236E13AEEBEFC7
:1027D00093F0EDEF93F0EEEF93F023802350D8B415
:1027E000F4EF93F0F6EF93F009EF94F02328D8A4D8
:1027F000FCEF93F0FEEF93F006EF94F0000E116EF5
:10280000000E126E000E136E000E146E138E11EF7A
:1028100094F0000E116E000E126E000E136E000E7C
:10282000146E1850800B1D1A18501824226E17AE03
:102830001CEF94F01EEF94F01FEF94F022802250D2
:10284000D8B425EF94F027EF94F03AEF94F02228D3
:10285000D8A42DEF94F02FEF94F037EF94F0000E02
:10286000156E000E166E000E176E000E186E178E87
:1028700042EF94F0000E156E000E166E000E176EED
:10288000000E186E2250D8B448EF94F04AEF94F03E
:1028900052EF94F02350D8A450EF94F052EF94F0FC
:1028A0005CEF94F0000E116E000E126E000E136EAF
:1028B000000E146E06EF96F0175011026F00CCFF59
:1028C00028F06F00D0FF29F028501E6E1F6A206A82
:1028D000216A2950246E256A266A276A1650120238
:1028E0006F00CCFF28F06F00D0FF29F028501E2683
:1028F000000E1F222022212229502426000E2522EC
:1029000026222722155013026F00CCFF28F06F00FB
:10291000D0FF29F028501E26000E1F22202221223F
:1029200029502426000E25222622272220C021F00D
:102930001FC020F01EC01FF01E6A155012026F004B
:10294000CCFF28F06F00D0FF29F028501E26295018
:102950001F22000E2022000E2122165011026F00AD
:10296000CCFF28F06F00D0FF29F028501E262950F8
:102970001F22000E2022000E212220C021F01FC0A5
:1029800020F01EC01FF01E6A155011026F00CCFF10
:1029900028F06F00D0FF29F028501E2629501F2252
:1029A000000E2022000E2122175012026F00CCFFD1
:1029B00028F06F00D0FF29F0285024262950252226
:1029C000000E2622000E2722165013026F00CCFFA5
:1029D00028F06F00D0FF29F0285024262950252206
:1029E000000E2622000E2722175013026F00CCFF84
:1029F00028F06F00D0FF29F02850196E29501A6E68
:102A00001B6A1C6A1BC01CF01AC01BF019C01AF00C
:102A1000196A195024261A5025221B5026221C50B0
:102A200027221EC019F01FC01AF020C01BF021C0C1
:102A30001CF0190E21EF95F0D8901C321B321A327F
:102A40001932E82E1CEF95F0195024261A50252231
:102A50001B5026221C50272220C021F01FC020F02E
:102A60001EC01FF01E6A225023C019F01A6A1926D0
:102A7000000E1A22820E1924286EFF0E1A20296ECB
:102A800057EF95F0D890243625362636273621AED6
:102A90004CEF95F04EEF95F04FEF95F02480D890E5
:102AA0001E361F36203621362806D8A0290626AE27
:102AB0005CEF95F05EEF95F042EF95F0000E226E20
:102AC00021AE65EF95F067EF95F08BEF95F0FF0E77
:102AD0001E14196EFF0E1F141A6EFF0E20141B6EAB
:102AE0007F0E21141C6E19501A101B101C10D8B424
:102AF0007CEF95F07EEF95F082EF95F0010E226E5F
:102B00008BEF95F024A087EF95F089EF95F08BEF90
:102B100095F07EEF95F02250D8B491EF95F093EFB9
:102B200095F0B7EF95F0010E2426000E25222622FF
:102B3000272227A09EEF95F0A0EF95F0B7EF95F034
:102B400024C019F025C01AF026C01BF027C01CF0C5
:102B50001C341C321B321A32193219C024F01AC02C
:102B600025F01BC026F01CC027F0284A292A29BEC0
:102B7000C2EF95F0295008E12828D8A0C2EF95F0BF
:102B8000C4EF95F0CEEF95F0000E246E000E256E8A
:102B9000800E266E7F0E276EFCEF95F029BEDBEFD0
:102BA00095F0295006E12804D8B0D9EF95F0DBEF75
:102BB00095F0E7EF95F0000E246E000E256E000EE6
:102BC000266E000E276E000E1D6EFCEF95F028C0DD
:102BD00023F0FF0E2416FF0E25167F0E2616000E7C
:102BE000271623A0F6EF95F0F8EF95F0F9EF95F0A2
:102BF000268ED8902330276E1D50271224C011F046
:102C000025C012F026C013F027C014F012002D507A
:102C1000800B3A6E2D502D24416E2CAE12EF96F0A3
:102C200014EF96F015EF96F041804150D8B41BEFA9
:102C300096F01DEF96F032EF96F04128D8A423EFDE
:102C400096F025EF96F02DEF96F0000E2A6E000E0E
:102C50002B6E000E2C6E000E2D6E2C8E000E2D6E27
:102C60003AEF96F0000E2A6E000E2B6E000E2C6EC0
:102C7000000E2D6E3150800B3A1A31503124426EC5
:102C800030AE45EF96F047EF96F048EF96F0428071
:102C90004250D8B44EEF96F050EF96F065EF96F0B4
:102CA0004228D8A456EF96F058EF96F060EF96F0D1
:102CB000000E2E6E000E2F6E000E306E000E316E66
:102CC000308E000E316E6DEF96F0000E2E6E000EFF
:102CD0002F6E000E306E000E316E2E502F10301001
:102CE0003110D8A476EF96F078EF96F090EF96F04A
:102CF000000E2A6E000E2B6E000E2C6E000E2D6E36
:102D0000800E2C127F0E2D123A502D122AC02AF05E
:102D10002BC02BF02CC02CF02DC02DF0D3EF97F052
:102D20004150D8A496EF96F098EF96F0A2EF96F067
:102D3000000E2A6E000E2B6E000E2C6E000E2D6EF5
:102D4000D3EF97F0425041C032F0336A325E000E4A
:102D5000335A7F0E32243B6E000E33203C6E2AC065
:102D600036F02BC037F02CC038F02DC039F0000EF3
:102D70002A6E000E2B6E000E2C6E000E2D6E000EB5
:102D80003D6E000E3E6E000E3F6E000E406E000E59
:102D9000426E03EF97F04250D8B4D1EF96F0D3EFE4
:102DA00096F0EAEF96F0D890363637363836393620
:102DB000D8902A362B362C362D3640AEE2EF96F0E0
:102DC000E4EF96F0E5EF96F02A80D8903D363E3657
:102DD0003F3640362E50365C2F50375830503858DA
:102DE00031503958D8A0F7EF96F0F9EF96F002EF8E
:102DF00097F0408C2E50365E2F50375A3050385A4C
:102E00003150395A422A190E426409EF97F00BEFFC
:102E100097F0CBEF96F03650371038103910D8B401
:102E200014EF97F016EF97F02EEF97F03D802EEF0E
:102E300097F0D8902A362B362C362D3640AE23EF1D
:102E400097F025EF97F026EF97F02A80D8903D363F
:102E50003E363F3640363B06D8A03C062CAE33EF1C
:102E600097F035EF97F019EF97F0000E426E40AEF5
:102E70003CEF97F03EEF97F062EF97F0FF0E3D14B6
:102E8000326EFF0E3E14336EFF0E3F14346E7F0E13
:102E90004014356E3250331034103510D8B453EF1F
:102EA00097F055EF97F059EF97F0010E426E62EFF1
:102EB00097F02AA05EEF97F060EF97F062EF97F03F
:102EC00055EF97F04250D8B468EF97F06AEF97F05B
:102ED0008EEF97F0010E2A26000E2B222C222D2297
:102EE0002DA075EF97F077EF97F08EEF97F02AC04F
:102EF00032F02BC033F02CC034F02DC035F0353417
:102F0000353234323332323232C02AF033C02BF011
:102F100034C02CF035C02DF03B4A3C2A3CBE99EF22
:102F200097F03C5008E13B28D8A099EF97F09BEF31
:102F300097F0A6EF97F0000E3C6E3B68000E2A6EED
:102F4000000E2B6E000E2C6E000E2D6E3CBEB3EFED
:102F500097F03C5006E13B04D8B0B1EF97F0B3EFE7
:102F600097F0C1EF97F0000E3C6E000E3B6E000E26
:102F70002A6E000E2B6E000E2C6E000E2D6E000EB3
:102F80003A6E3BC041F041A0C8EF97F0CAEF97F00E
:102F9000CDEF97F02C8ECEEF97F02C9ED89041304D
:102FA0002D6E84EF96F012002B0E036EFC0E046E55
:102FB000C9ECB2F0C10E0001EC6F010EED6F000E16
:102FC0000101C16F410EC26F270EC36F400E000199
:102FD000FB6F030EFC6FECC018F0EDC019F0FCC0E5
:102FE0001AF01B6AFB5113ECB2F0710E036EFB0E6C
:102FF000046EC9ECB2F0050E0101C16F0D0EC26F77
:103000001B0EC36F400E0001FB6FC10EEC6F010E73
:10301000ED6F030EFC6FECC018F0EDC019F0FCC0B2
:103020001AF01B6AFB5113ECB2F0510E036EFA0E4C
:10303000046EC9ECB2F0060E0101C16F800EC26FC2
:10304000010EC36F400E0001FB6FC10EEC6F010E4D
:10305000ED6F030EFC6FECC018F0EDC019F0FCC072
:103060001AF01B6AFB5113ECB2F04B0E036EF90E13
:10307000046EC9ECB2F0070E0101C16F270EC26FDA
:10308000100EC36F400E0001FB6FC10EEC6F010EFE
:10309000ED6F030EFC6FECC018F0EDC019F0FCC032
:1030A0001AF01B6AFB5113ECB2F0400E0001FB6FEB
:1030B000000E0101C16F000EC26FC10E0001EC6F66
:1030C000010EED6F040E186EECC019F0EDC01AF091
:1030D000000E1C6E030E1B6EFB5122ECAFF00101C3
:1030E000C1510001E36FE26B0101C2510001E22511
:1030F000FD6F0101000E0001E321FE6F580EC96F44
:10310000020ECA6FF00ECB6FFC0ECC6FFDC0CDF07F
:10311000FEC0CEF01EECB3F0580E036E020E046E2D
:1031200040ECB1F0400E0001FB6F000E0101C16FD9
:10313000000EC26FC10E0001EC6F010EED6F070EA5
:10314000186EECC019F0EDC01AF0000E1C6E030EE4
:103150001B6EFB5122ECAFF00101C1510001E36F86
:10316000E26B0101C2510001E225FD6F0101000E79
:103170000001E321FE6F170E156EB70E166E510E8D
:10318000176E3F0E186EFDC003F0FEC004F0056A16
:10319000066A000EA8EC9FF003C011F004C012F004
:1031A00005C013F006C014F0E0EC93F011C02AF053
:1031B00012C02BF013C02CF014C02DF0000E2E6E98
:1031C000000E2F6E000E306E470E316E07EC96F03B
:1031D0002AC046F12BC047F12CC048F12DC049F15F
:1031E000580E0001C96F020ECA6F0B0ECB6FFC0E9A
:1031F000CC6F46C1CDF047C1CEF048C1CFF049C138
:10320000D0F01EECB3F0580E036E020E046E40ECCC
:10321000B1F0400E0001FB6F000E0101C16F000E06
:10322000C26F000EC36FC10E0001EC6F010EED6F97
:10323000FE0E186EECC019F0EDC01AF0000E1C6EF8
:10324000030E1B6EFB5122ECAFF00101C1510001D6
:10325000E36FE26B0101C2510001E225FD6F010144
:10326000000E0001E321FE6F580EC96F020ECA6FF7
:10327000620ECB6FFD0ECC6FFDC0CDF0FEC0CEF068
:103280001EECB3F0580E036E020E046E40ECB1F06B
:10329000400E0001FB6F000E0101C16F000EC26FF6
:1032A000000EC36FC10E0001EC6F010EED6FFF0E3B
:1032B000186EECC019F0EDC01AF0000E1C6E030E73
:1032C0001B6EFB5122ECAFF00101C1510001E36F15
:1032D000E26B0101C2510001E225FD6F0101000E08
:1032E0000001E321FE6F580EC96F020ECA6F7D0EFA
:1032F000CB6FFD0ECC6FFDC0CDF0FEC0CEF01EEC4E
:10330000B3F0580E036E020E046E40ECB1F0BE0E28
:10331000036EFB0E046EC9ECB2F0120020C038F050
:1033200021C039F022C03AF023C03BF024C03CF069
:1033300025C03DF026C03EF027C03FF03FBEA3EFC2
:1033400099F0A6EF99F0010EA7EF99F0000E366EF6
:10335000376A36503710D8B4B0EF99F0B2EF99F021
:10336000C2EF99F03F1E3E1E3D1E3C1E3B1E3A1E04
:10337000391E386C000E39223A223B223C223D2273
:103380003E223F220001E9BFC8EF99F0CAEF99F051
:10339000CBEF99F0EA93E9BFD8EF99F0E95106E154
:1033A000E805D8B0D6EF99F0D8EF99F0DEEF99F0B4
:1033B000000E336E010E326EE2EF99F0E8C032F08B
:1033C000E9C033F068C134F069C135F036503710C8
:1033D000D8A4EDEF99F0EFEF99F0F6EF99F0EAA5A8
:1033E000F4EF99F0F6EF99F0F9EF99F03406D8A0E0
:1033F0003506000E416E4F0E406E000E0201576FF3
:103400007EEF9AF04006D8A04106080E4024D96EFF
:10341000020E4120DA6E38C003F039C004F03AC021
:1034200005F03BC006F03CC007F03DC008F03EC0D0
:1034300009F03FC00AF00A0E0B6E000E0C6E000E73
:103440000D6E000E0E6E000E0F6E000E106E000E52
:10345000116E000E126ED9ECA2F003C028F004C069
:1034600029F005C02AF006C02BF007C02CF008C0D8
:103470002DF009C02EF00AC02FF028C015F02AC088
:1034800016F0DFECB4F01550300FDF6E3206D8A026
:1034900033063406D8A0350638C003F039C004F02E
:1034A0003AC005F03BC006F03CC007F03DC008F054
:1034B0003EC009F03FC00AF00A0E0B6E000E0C6E03
:1034C000000E0D6E000E0E6E000E0F6E000E106ED2
:1034D000000E116E000E126E56ECA1F003C038F013
:1034E00004C039F005C03AF006C03BF007C03CF01C
:1034F00008C03DF009C03EF00AC03FF041BE89EF70
:103500009AF0415008E14004D8A089EF9AF08BEF7F
:103510009AF0BCEF9AF0385039103A103B103C103A
:103520003D103E103F10D8A498EF9AF09AEF9AF011
:1035300002EF9AF033BEA7EF9AF0335006E132045F
:10354000D8B0A5EF9AF0A7EF9AF002EF9AF035BE47
:10355000B2EF9AF0355008E13404D8A0B2EF9AF0F7
:10356000B4EF9AF0BCEF9AF00001EAB3BAEF9AF028
:10357000BCEF9AF002EF9AF036503710D8A4C3EFA0
:103580009AF0C5EF9AF0CDEF9AF00001EAA5CBEFE3
:103590009AF0CDEF9AF0ECEF9AF04006D8A04106F1
:1035A00036503710D8A4D7EF9AF0D9EF9AF0DFEF62
:1035B0009AF0000E316E2B0E306EE3EF9AF0000E93
:1035C000316E2D0E306E080E4024D96E020E412051
:1035D000DA6E6000C3F0DFFF1EC013F01FC014F0EE
:1035E000080E4024156E020E4120166E34C017F0EE
:1035F00035C018F0A7ECAAF013C01EF014C01FF0DD
:1036000012000001E9BF07EF9BF009EF9BF00AEF02
:103610009BF0EA93E9BF17EF9BF0E95106E1E8055B
:10362000D8B015EF9BF017EF9BF01DEF9BF0000E4D
:10363000326E010E316E21EF9BF0E8C031F0E9C02F
:1036400032F068C133F069C134F0EAA92AEF9BF087
:103650002CEF9BF030EF9BF0FE0E3326FF0E342252
:1036600020C035F021C036F022C037F023C038F03A
:1036700024C039F025C03AF026C03BF027C03CF00A
:10368000000E3E6E4F0E3D6E000E0201576FE3EFCF
:103690009BF03D06D8A03E060F0E35143F6E406AE3
:1036A00040BE5CEF9BF0405009E10A0E3F5CD8A0A1
:1036B0005CEF9BF05EEF9BF066EF9BF0570E3F24B4
:1036C0003F6E000E4020406E6CEF9BF0300E3F24AA
:1036D0003F6E000E4020406EBF0E296EFF0E2A6E18
:1036E00028502B6E2C6A29502B262A502C222C5025
:1036F00007E11A0E2B5CD8B080EF9BF082EF9BF0B5
:10370000A5EF9BF09F0E296EFF0E2A6E200E3F1034
:103710002B6E000E40102C6E29502B262A502C2286
:103720002C5007E11A0E2B5CD8B099EF9BF09BEF61
:103730009BF0A5EF9BF03FC009F040C00AF09BEC66
:10374000B4F009C03FF00AC040F0080E3D24D96E25
:10375000020E3E20DA6E6000FFF0DFFF3106D8A0D7
:1037600032063306D8A0340635C029F036C02AF018
:1037700037C02BF038C02CF039C02DF03AC02EF0F5
:103780003BC02FF03CC030F0050ED0EF9BF0D8903E
:1037900030322F322E322D322C322B322A32293235
:1037A000E82EC7EF9BF029C035F02AC036F02BC0B9
:1037B00037F02CC038F02DC039F02EC03AF02FC0B1
:1037C0003BF030C03CF03EBEEFEF9BF03E5009E1D5
:1037D000020E3D5CD8A0EFEF9BF0F1EF9BF022EFE3
:1037E0009CF0355036103710381039103A103B1015
:1037F0003C10D8A4FEEF9BF000EF9CF049EF9BF04B
:1038000032BE0DEF9CF0325006E13104D8B00BEF20
:103810009CF00DEF9CF049EF9BF034BE18EF9CF04C
:10382000345008E13304D8A018EF9CF01AEF9CF054
:1038300022EF9CF00001EAB320EF9CF022EF9CF015
:1038400049EF9BF00001EAA928EF9CF02AEF9CF0D9
:1038500041EF9CF03D06D8A03E06080E3D24D96EEF
:10386000020E3E20DA6E6000A3F0DFFF3D06D8A016
:103870003E06080E3D24D96E020E3E20DA6E300E52
:10388000DF6E1EC013F01FC014F0080E3D24156E2D
:10389000020E3E20166E33C017F034C018F0A7ECAD
:1038A000AAF013C01EF014C01FF01200000E000199
:1038B000F06F040EF16F6000C3F3D9FF6000C7F32F
:1038C000DAFF000EDF6E3D017599738F000E000167
:1038D000E76F020EE66FE651AAECB5F00009D8B426
:1038E00074EF9CF076EF9CF080EF9DF00001E735DF
:1038F000E731E26FE631FD6FE2C0FEF0F0C0C9F0E3
:10390000F1C0CAF0430ECB6FFB0ECC6FE6C0CDF01A
:10391000E7C0CEF0FDC0CFF0FEC0D0F01EECB3F09B
:1039200021EF9DF0F0C011F0F1C012F0970E136E70
:10393000FD0E146EE6ECB6F078EF9DF0580E036EB7
:10394000020E046E430E056EFF0E066ECEECB0F056
:10395000F0C003F0F1C004F09DECB2F003C0E4F05D
:1039600004C0E5F00001E451F025076EE551F121B6
:10397000086E580E096E020E0A6EAFECB1F078EFC9
:103980009DF0F0C011F0F1C012F0310E136EFF0E79
:10399000146EE6ECB6F078EF9DF0F0C011F0F1C0D7
:1039A00012F00C0E136EFF0E146EE6ECB6F078EF0C
:1039B0009DF0F0C011F0F1C012F0910E136EFF0EE9
:1039C000146EE6ECB6F078EF9DF0F0C011F0F1C0A7
:1039D00012F0520E136EFE0E146EE6ECB6F078EF97
:1039E0009DF0F0C011F0F1C012F0740E136EFF0ED6
:1039F000146EE6ECB6F078EF9DF0F0C011F0F1C077
:103A000012F0B60E136EFF0E146EE6ECB6F078EF01
:103A10009DF0F0C011F0F1C012F02B0E136EFD0EF0
:103A2000146EE6ECB6F078EF9DF0F0C011F0F1C046
:103A300012F09E0E136EFF0E146EE6ECB6F078EFE9
:103A40009DF0FDC0E2F0FEC0E3F00001E351000A8A
:103A5000D8B42DEF9DF015EF9DF0E251200AD8B4B7
:103A600092EF9CF0010AD8B492EF9CF0030AD8B40C
:103A700092EF9CF0010AD8B492EF9CF0040AD8B4FB
:103A800092EF9CF00F0AD8B49EEF9CF0010AD8B4D4
:103A90009EEF9CF0030AD8B49EEF9CF01D0AD8B4A8
:103AA000C1EF9CF00F0AD8B4CDEF9CF0010AD8B456
:103AB000CDEF9CF0030AD8B4CDEF9CF0010AD8B446
:103AC000CDEF9CF0070AD8B4D9EF9CF07C0AD8B4AB
:103AD000E5EF9CF0170AD8B4F1EF9CF03F0AD8B498
:103AE000FDEF9CF0C80AD8B409EF9DF015EF9DF0EA
:103AF000F0C003F0F1C004F040ECB1F024ECB6F0FB
:103B0000020E0001E625E66F000EE721E76FE7BF32
:103B100093EF9DF0E75109E1FC0EE65DD8A093EF2D
:103B20009DF095EF9DF06BEF9CF03D01739F7589C3
:103B300024ECB6F03D01738F12003EC153F03FC13B
:103B400054F040C155F041C156F043C053F044C059
:103B500054F045C055F046C056F0810E476EFF0E3A
:103B6000486E53C049F054C04AF055C04BF056C09F
:103B70004CF0180EC1EF9DF0D8904C324B324A32C7
:103B80004932E82EBCEF9DF049504724516E000E9B
:103B90004820526E52BED6EF9DF0525009E1170EEA
:103BA000515CD8A0D6EF9DF0D8EF9DF0E2EF9DF0EC
:103BB00043C043F044C044F045C045F046C046F021
:103BC000A5EF9EF052BEE7EF9DF0E9EF9DF059EFB3
:103BD0009EF051C047F0FF0E486EFF0E496E7F0EFB
:103BE0004A6E000E4B6E4766F8EF9DF000EF9EF0B8
:103BF0004B344B324A3249324832472EF3EF9DF074
:103C000048C04DF049C04EF04AC04FF04BC050F094
:103C10004D505314476E4E505414486E4F50551427
:103C2000496E505056144A6E4750481049104A1079
:103C3000D8A41DEF9EF01FEF9EF021EF9EF0D8EF6D
:103C40009DF053C047F054C048F055C049F056C0ED
:103C50004AF0200E31EF9EF0D8904A324932483275
:103C60004732E82E2CEF9EF04750481049104A107A
:103C7000D8B43DEF9EF03FEF9EF047EF9EF04D50E1
:103C800053264E5054224F505522505056224D1C10
:103C9000476E4E1C486E4F1C496E501C4A6E475072
:103CA000531648505416495055164A5056169DEF13
:103CB0009EF053C047F054C048F055C049F056C07C
:103CC0004AF0200E69EF9EF0D8904A3249324832CD
:103CD0004732E82E64EF9EF04750481049104A10D2
:103CE000D8A475EF9EF077EF9EF081EF9EF0000E66
:103CF000536E000E546E000E556E000E566E9DEF04
:103D00009EF0D8905334476E5434486E5534496E03
:103D100056344A6E4750481049104A10D8B493EFB1
:103D20009EF095EF9EF09DEF9EF0000E536E000EFC
:103D3000546E800E556EBF0E566E53C043F054C085
:103D400044F055C045F056C046F012000001E9BFEE
:103D5000ACEF9EF0AEEF9EF0AFEF9EF0EA93E9BFBE
:103D6000BCEF9EF0E95106E1E805D8B0BAEF9EF04D
:103D7000BCEF9EF0C2EF9EF0000E316E010E306E71
:103D8000C6EF9EF0E8C030F0E9C031F068C132F013
:103D900069C133F020C034F021C035F022C036F0C4
:103DA00023C037F024C038F025C039F026C03AF0DF
:103DB00027C03BF0000E3D6E4F0E3C6E000E020120
:103DC000576F59EF9FF03C06D8A03D06080E3C24E3
:103DD000D96E020E3D20DA6E34C003F035C004F017
:103DE00036C005F037C006F038C007F039C008F01B
:103DF0003AC009F03BC00AF00A0E0B6E000E0C6EC2
:103E0000000E0D6E000E0E6E000E0F6E000E106E88
:103E1000000E116E000E126E79ECA9F003C028F0AE
:103E200004C029F005C02AF006C02BF007C02CF012
:103E300008C02DF009C02EF00AC02FF02850300F16
:103E4000DF6E3006D8A031063206D8A0330634C063
:103E500003F035C004F036C005F037C006F038C0B6
:103E600007F039C008F03AC009F03BC00AF00A0E6A
:103E70000B6E000E0C6E000E0D6E000E0E6E000E20
:103E80000F6E000E106E000E116E000E126E95EC8D
:103E9000A8F003C034F004C035F005C036F006C009
:103EA00037F007C038F008C039F009C03AF00AC04E
:103EB0003BF03C503D10D8B460EF9FF062EF9FF0B4
:103EC00093EF9FF0345035103610371038103910FA
:103ED0003A103B10D8A46FEF9FF071EF9FF0E3EF23
:103EE0009EF031BE7EEF9FF0315006E13004D8B035
:103EF0007CEF9FF07EEF9FF0E3EF9EF033BE89EF03
:103F00009FF0335008E13204D8A089EF9FF08BEF87
:103F10009FF093EF9FF00001EAB391EF9FF093EFD2
:103F20009FF0E3EF9EF01EC013F01FC014F0080EC8
:103F30003C24156E020E3D20166E32C017F033C0C1
:103F400018F0A7ECAAF013C01EF014C01FF0120066
:103F50000B6E0B50D8B4AFEF9FF0B1EF9FF0D3EFE3
:103F60009FF006BEB8EF9FF0B6EF9FF0D3EF9FF043
:103F700003C007F004C008F005C009F006C00AF04D
:103F8000071E081E091E0A1E072A000E0822092203
:103F90000A2207C00DF008C00EF009C00FF00AC0D9
:103FA00010F0DBEF9FF003C00DF004C00EF005C071
:103FB0000FF006C010F00350041005100610D8A42E
:103FC000E4EF9FF0E6EF9FF0F0EF9FF0000E036E3E
:103FD000000E046E000E056E000E066E81EFA0F05E
:103FE000960E0C6EFAEF9FF00C2AD89010320F321A
:103FF0000E320D32000E0D14076E000E0E14086EF8
:10400000000E0F14096EFE0E10140A6E07500810F1
:1040100009100A10D8A40FEFA0F011EFA0F0F4EFF0
:104020009FF01FEFA0F00C2A010E0D26000E0E22AD
:104030000F221022D89010320F320E320D32000EA5
:104040000D14076E000E0E14086E000E0F14096E8C
:10405000FF0E10140A6E0750081009100A10D8A499
:1040600034EFA0F036EFA0F013EFA0F03EEFA0F099
:104070000C06D8900D360E360F3610360FBE43EFB5
:10408000A0F045EFA0F04DEFA0F0020E0C604BEF5A
:10409000A0F04DEFA0F038EFA0F00CB052EFA0F080
:1040A00054EFA0F055EFA0F00F9ED8900C320CC04A
:1040B00007F0086A096A0A6A07C00AF0096A086A0A
:1040C000076A07500D1208500E1209500F120A50BD
:1040D00010120B50D8B46FEFA0F071EFA0F079EF91
:1040E000A0F006BE78EFA0F076EFA0F079EFA0F098
:1040F000108E0DC003F00EC004F00FC005F010C00C
:1041000006F0120020EED5F110EE11F0060E6F0051
:104110006FFFE3FFE806FBE20EC01CF00FC01DF0CE
:104120001C501D10D8A497EFA0F099EFA0F09DEFC0
:10413000A0F0110E1C6E000E1D6E1CC003F01DC001
:1041400004F09DECB2F003C020F004C021F0E8C000
:104150001EF0E9C01FF01FBEB0EFA0F0B2EFA0F05C
:10416000C7EFA0F020501E5C1F50800A106E215037
:10417000800A1058D8A0BFEFA0F0C1EFA0F0C3EFA5
:10418000A0F0C7EFA0F01EC020F01FC021F020C09B
:104190001EF021C01FF068C11AF069C11BF00001B8
:1041A000EAB1D5EFA0F0D7EFA0F0F4EFA0F0E5EF83
:1041B000A0F0000E046E200E036E0CC005F00DC0C2
:1041C00006F00DECA9F0204A212A1A50205C21505B
:1041D000800A106E1B50800A1058D8A0F2EFA0F091
:1041E000F4EFA0F0D9EFA0F0000E196E000E186EDB
:1041F0001DEFA1F0600073F0F6FF600077F0F7FFAD
:10420000000EF86E1F0EF76403D00800F55007D0BB
:104210006F00DBFFE9FF6F00DFFFEAFFEF50106E7A
:104220001050036E046A0CC005F00DC006F00DECD2
:10423000A9F01C4A1D2A184A192A1E50185C195048
:10424000800A106E1F50800A1058D8A02AEFA1F0E3
:104250002CEFA1F0FAEFA0F00001EAA132EFA1F0FB
:1042600034EFA1F051EFA1F042EFA1F0000E046E87
:10427000200E036E0CC005F00DC006F00DECA9F089
:10428000204A212A1A50205C2150800A106E1B50AF
:10429000800A1058D8A04FEFA1F051EFA1F036EFEF
:1042A000A1F020C00CF021C00DF01200000E146E21
:1042B00012BE5FEFA1F05DEFA1F071EFA1F0121E51
:1042C000111E101E0F1E0E1E0D1E0C1E0B6C000E5E
:1042D0000C220D220E220F22102211221222010E78
:1042E000146E0ABE78EFA1F076EFA1F08AEFA1F08C
:1042F0000A1E091E081E071E061E051E041E036C4C
:10430000000E0422052206220722082209220A2280
:10431000010E141A20EE15F0070EDE6AE806FDE223
:104320000B500C100D100E100F1010101110121059
:10433000D8B49DEFA1F09FEFA1F0F1EFA1F0010E35
:10434000136EADEFA1F0D8900B360C360D360E364D
:104350000F36103611361236132A12AEB2EFA1F014
:10436000B4EFA1F0A3EFA1F0D890153616361736AA
:10437000183619361A361B361C360B50035C0C5097
:1043800004580D5005580E5006580F50075810503D
:1043900008581150095812500A58D8A0D2EFA1F06D
:1043A000D4EFA1F0E5EFA1F00B50035E0C50045ADE
:1043B0000D50055A0E50065A0F50075A1050085A01
:1043C0001150095A12500A5A1580D89012321132DF
:1043D00010320F320E320D320C320B32132EB4EF7C
:1043E000A1F01450D8B4F7EFA1F0F9EFA1F009EF64
:1043F000A2F01C1E1B1E1A1E191E181E171E161EAA
:10440000156C000E16221722182219221A221B22BE
:104410001C2215C003F016C004F017C005F018C028
:1044200006F019C007F01AC008F01BC009F01CC044
:104430000AF01200000E136E000E126E000E116EC6
:10444000000E106E26EFA2F00A4A0B2A60002BF035
:10445000F6FF60002FF0F7FF000EF86E0800F55031
:10446000200AD8B436EFA2F038EFA2F024EFA2F081
:10447000F70E0C6EFF0E0D6E60002BF0F6FF600065
:104480002FF0F7FF000EF86E0800F5500E6E0F6A61
:104490000C500E260D500F220F5009E1050E0E5C38
:1044A000D8A055EFA2F057EFA2F024EFA2F061EFF1
:1044B000A2F0000E116E010E106E0A4A0B2A9EEF3A
:1044C000A2F060002BF0F6FF60002FF0F7FF000E67
:1044D000F86E0800F5500C6E0D6A0D50000AD8B445
:1044E00074EFA2F09EEFA2F00C502B0AD8B45DEF4F
:1044F000A2F0060AD8B459EFA2F09EEFA2F012C0C3
:1045000003F013C004F0000E066E0A0E056E95EC63
:10451000B6F060002BF0F6FF60002FF0F7FF000E02
:10452000F86E0800F550035E000E045A300E0324A6
:10453000126E000E0420136E5DEFA2F0D00E0C6E12
:10454000FF0E0D6E60002BF0F6FF60002FF0F7FFFE
:10455000000EF86E0800F5500E6E0F6A0C500E2615
:104560000D500F220F5009E10A0E0E5CD8A0BBEFD0
:10457000A2F0BDEFA2F07FEFA2F010501110D8A46E
:10458000C4EFA2F0C6EFA2F0D4EFA2F012C00CF07C
:1045900013C00DF00C1E0D1E0C4A0D2A0CC00AF0A3
:1045A0000DC00BF0D8EFA2F012C00AF013C00BF050
:1045B0001200000E146E0ABEE2EFA2F0E0EFA2F0CD
:1045C000F4EFA2F00A1E091E081E071E061E051E95
:1045D000041E036C000E0422052206220722082274
:1045E00009220A22010E146E12BEFBEFA2F0F9EFAF
:1045F000A2F00BEFA3F0121E111E101E0F1E0E1EB6
:104600000D1E0C1E0B6C000E0C220D220E220F2212
:104610001022112212220B500C100D100E100F1030
:10462000101011101210D8B418EFA3F01AEFA3F065
:1046300062EFA3F0010E136E28EFA3F0D8900B36B3
:104640000C360D360E360F36103611361236132A4A
:1046500012AE2DEFA3F02FEFA3F01EEFA3F00B503F
:10466000035C0C5004580D5005580E5006580F505E
:104670000758105008581150095812500A58D8A01D
:1046800044EFA3F046EFA3F056EFA3F00B50035E08
:104690000C50045A0D50055A0E50065A0F50075A26
:1046A0001050085A1150095A12500A5AD890123212
:1046B000113210320F320E320D320C320B32132EF9
:1046C0002FEFA3F01450D8B468EFA3F06AEFA3F073
:1046D0007AEFA3F00A1E091E081E071E061E051EFD
:1046E000041E036C000E0422052206220722082263
:1046F00009220A2203C003F004C004F005C005F03B
:1047000006C006F007C007F008C008F009C009F0AD
:104710000AC00AF0120003C00AF004C00BF005C082
:104720000CF006C00DF00706D8A00806072806E121
:104730000828D8A49EEFA3F0A0EFA3F0ADEFA3F05C
:10474000000E046E000E036E33EFA4F00A4A0B2A2B
:104750000C4A0D2A0706D8A0080660002BF0F6FFC9
:1047600060002FF0F7FF000EF86E1F0EF76403D005
:104770000800F55007D06F00DBFFE9FF6F00DFFF97
:10478000EAFFEF500009D8B4C8EFA3F0CAEFA3F0D6
:104790000EEFA4F0600033F0F6FF600037F0F7FF93
:1047A000000EF86E0800F5500009D8B4DAEFA3F057
:1047B000DCEFA3F00EEFA4F007500810D8B4E3EF3D
:1047C000A3F0E5EFA3F00EEFA4F0600033F0F6FFE6
:1047D000600037F0F7FF000EF86E08006F00D4FF9E
:1047E00009F060002BF0F6FF60002FF0F7FF000EDD
:1047F000F86E1F0EF76403D00800F55007D06F0065
:10480000DBFFE9FF6F00DFFFEAFFEF500918D8B4C4
:104810000CEFA4F00EEFA4F0A6EFA3F060002BF0D5
:10482000F6FF60002FF0F7FF000EF86E1F0EF76422
:1048300003D00800F55007D06F00DBFFE9FF6F00E1
:10484000DFFFEAFFEF50096E600033F0F6FF600013
:1048500037F0F7FF000EF86E0800F550095C036EA4
:10486000046AD8A004061200400EDEECAEF0030E7F
:10487000256E080E246E770EE82EFED7242EFCD768
:10488000252EFAD700F0000E276E000E266E2204A9
:104890002310D8A44EEFA4F050EFA4F058EFA4F0EA
:1048A0003A0E036EF60E046EC9ECB2F024ECB6F0CC
:1048B000000E296E000E286E22042310D8A463EF88
:1048C000A4F065EFA4F096EFA4F028502910D8B416
:1048D0006CEFA4F06EEFA4F096EFA4F0070E28148E
:1048E000246E000E2914256E24502510D8A47BEFC9
:1048F000A4F07DEFA4F096EFA4F026C024F027C02A
:1049000025F0D89024362536D89024362536D890F0
:10491000243625363A0E2424036EF60E2520046E26
:10492000C9ECB2F0264A272A24ECB6F0070E282458
:10493000F66EF50E2920F76EF86A000EF8220800D0
:10494000F5509AECAEF022042310D8A4AAEFA4F0FC
:10495000ACEFA4F0BBEFA4F0070E2824F66EF50E22
:104960002920F76EF86A000EF8220800F55032ECA4
:10497000B4F024ECB6F0284A292A295009E1400E67
:10498000285CD8A0C6EFA4F0C8EFA4F05CEFA4F0B8
:10499000800EDEECAEF0D00E246ECA0EE82EFED7EE
:1049A000242EFCD71200F80E036EFF0E046EC9EC25
:1049B000B2F0000E1F6E300E07ECAEF0680E236EE4
:1049C000E40EE82EFED7232EFCD700D0320E2FECBB
:1049D000B7F0000E1F6E300E07ECAEF0150E236E12
:1049E000C60EE82EFED7232EFCD700D0330E2FECB8
:1049F000B7F0000E1F6E300E07ECAEF0150E236EF2
:104A0000C60EE82EFED7232EFCD700D0340E2FEC96
:104A1000B7F0000E1F6E250E07ECAEF0150E236EDC
:104A2000C60EE82EFED7232EFCD700D0350E2FEC75
:104A3000B7F0010E1F6E280E07ECAEF0150E236EB8
:104A4000C60EE82EFED7232EFCD700D0360E2FEC54
:104A5000B7F0010E1F6E080E07ECAEF0150E236EB8
:104A6000C60EE82EFED7232EFCD700D0370E2FEC33
:104A7000B7F0010E1F6E010E07ECAEF0030E246EB0
:104A8000080E236E770EE82EFED7232EFCD7242E99
:104A9000FAD700F0380E2FECB7F0010E1F6E060E9D
:104AA00007ECAEF0150E236EC60EE82EFED7232EB1
:104AB000FCD700D0390E2FECB7F0010E1F6E0C0E94
:104AC00007ECAEF0150E236EC60EE82EFED7232E91
:104AD000FCD700D04F0E2FECB7F04B0E2FECB7F0F9
:104AE00012008FECB7F00009D8B479EFA5F07BEF96
:104AF000A5F0B7EFA5F088EFA5F0E6ECB7F003EF6F
:104B0000A6F03CECB8F003EFA6F0000E03EFA6F021
:104B100018C10EF019C10FF020EE09F102D89BEF79
:104B2000A5F00500FA6EDE50FD6EDE50FE6EDE5022
:104B3000FF6EFA501200106E116A1150000AD8B4BC
:104B4000A4EFA5F085EFA5F01050010AD8B485EFC9
:104B5000A5F0030AD8B47DEFA5F0010AD8B481EF1F
:104B6000A5F0070AD8B485EFA5F085EFA5F084EC91
:104B7000B7F00009D8B4BFEFA5F0C1EFA5F002EF80
:104B8000A6F001012951030B0009D8B4CAEFA5F022
:104B9000CCEFA5F0D8EFA5F0010E106E2951030B54
:104BA000116E1050115E29511118FC0B1118296F4C
:104BB00060008FF4D9FF600093F4DAFFDF50146EC9
:104BC000234B242B2507D8A0260725512611D8A42E
:104BD000ECEFA5F0EEEFA5F0F6EFA5F065ECAFF089
:104BE000106E1050126E136AFAEFA5F0000E136EDD
:104BF000030E126E12C015F01450F9ECB7F01550F8
:104C000003EFA6F0030E1200270E0001FB6F020E49
:104C1000DEECAEF0090E0001E36F1E0EE26FE40E53
:104C2000E82EFED7E22FFCD7E32FFAD700F0010ED3
:104C3000266E7D0E276EFE0E286E010E95ECA7F0F7
:104C4000000E0201586F580E0001C96F020ECA6FA4
:104C50001F0ECB6FFF0ECC6F9AC1CDF09BC1CEF073
:104C60001EECB3F0010E276E580E286E020E296E50
:104C7000020EAAECB6F0000E0201586F580E0001A9
:104C8000C96F020ECA6F640ECB6FFF0ECC6F74C17A
:104C9000CDF075C1CEF076C1CFF077C1D0F01EEC6B
:104CA000B3F0010E276E580E286E020E296E030E09
:104CB000AAECB6F0000E0201586F580E0001C96F41
:104CC000020ECA6F3C0ECB6FFE0ECC6F4AC1CDF008
:104CD0004BC1CEF04CC1CFF04DC1D0F04EC1D1F0A0
:104CE0004FC1D2F050C1D3F051C1D4F01EECB3F09B
:104CF0000101B805D8A47FEFA6F081EFA6F086EFFA
:104D0000A6F0410E02016A6F4C0E6B6F010E276E0A
:104D1000580E286E020E296E040EAAECB6F0120090
:104D2000053406340C6E0C50D8A499EFA6F09BEF16
:104D3000A6F0A5EFA6F0000E036E000E046E000EA6
:104D4000056E000E066E12EFA7F003C007F004C058
:104D500008F005C009F006C00AF0200EB5EFA6F075
:104D6000D8900A32093208320732E82EB0EFA6F0A6
:104D700007500B6E058EFF0E0316FF0E0416FF0E76
:104D80000516000E0616960E0C5E0CBECCEFA6F0B5
:104D9000CAEFA6F0E2EFA6F00C50800A970FD8B049
:104DA000D4EFA6F0D6EFA6F0D8EFA6F09BEFA6F0D2
:104DB000D89006320532043203320C3ED8EFA6F00A
:104DC000FAEFA6F01F0E0C64E8EFA6F0EAEFA6F0EB
:104DD000F2EFA6F09BEFA6F0D89003360436053626
:104DE00006360C060C50D8A4F8EFA6F0FAEFA6F0A1
:104DF000ECEFA6F00B50D8B400EFA7F002EFA7F04D
:104E00000AEFA7F0061E051E041E036C000E042206
:104E10000522062203C003F004C004F005C005F01B
:104E200006C006F01200000E2A14326E000E2B147B
:104E3000336E800E2C14346E7F0E2D14356E32506E
:104E4000331034103510D8A428EFA7F02AEFA7F0BC
:104E500032EFA7F0000E2A6E000E2B6E000E2C6EA5
:104E6000000E2D6E000E2E14326E000E2F14336EB7
:104E7000800E3014346E7F0E3114356E3250331084
:104E800034103510D8A447EFA7F049EFA7F051EF41
:104E9000A7F0000E2E6E000E2F6E000E306E000E6C
:104EA000316E2DAE56EFA7F058EFA7F061EFA7F0E7
:104EB0002A6C2B1ED8B02B2A2C1ED8B02C2A800E80
:104EC0002D5631AE66EFA7F068EFA7F071EFA7F0AF
:104ED0002E6C2F1ED8B02F2A301ED8B0302A800E4C
:104EE0003156000E2A1A000E2B1A000E2C1A800EB4
:104EF0002D1A000E2E1A000E2F1A000E301A800ED8
:104F0000311A2E502A5C2F502B5830502C583150CB
:104F10002D58D8B08EEFA7F090EFA7F093EFA7F041
:104F2000D89094EFA7F0D8801200456E27C003F008
:104F300028C004F09DECB2F003C043F004C044F07C
:104F400044BEAEEFA7F0445007E1150E435CD8B065
:104F5000ACEFA7F0AEEFA7F015EFA8F02E0E036EA2
:104F6000000E046E27C005F028C006F0CEECB0F0AD
:104F7000000E426E43505C5C296E44505D582A6EB0
:104F800026502B6E2C6A29502B5C2C50800A2D6EDB
:104F90002A50800A2D58D8A0D0EFA7F0D2EFA7F062
:104FA000D4EFA7F0010E266E4504D8A4DAEFA7F0DF
:104FB000DCEFA7F0E0EFA7F026507F0FDEECAEF0BD
:104FC000020E4518D8A4E7EFA7F0E9EFA7F0EDEF40
:104FD000A7F02650BF0FDEECAEF0030E4518D8A4A4
:104FE000F4EFA7F0F6EFA7F0FAEFA7F02650930F33
:104FF000DEECAEF0040E4518D8A401EFA8F003EFE4
:10500000A8F007EFA8F02650D30FDEECAEF0150E97
:10501000296EC60EE82EFED7292EFCD700D02E0E04
:10502000216E000E226EE4ECB1F0120042C10DF0D0
:1050300043C10EF044C10FF045C110F003C00DF0A4
:1050400004C00EF005C00FF006C010F00DC007F050
:105050000EC008F00FC009F010C00AF0180E36EFAD
:10506000A8F0D8900A32093208320732E82E31EF20
:10507000A8F007500B6E0C6A0B500C10D8A443EF2D
:10508000A8F045EFA8F065EFA8F0D8900D34076EB2
:105090000E34086E0F34096E10340A6E0750081073
:1050A00009100A10D8A457EFA8F059EFA8F05FEF45
:1050B000A8F0000E046E020E036E94EFA8F0000E2E
:1050C000046E030E036E94EFA8F00B280C10D8A406
:1050D0006CEFA8F06EEFA8F090EFA8F00DC007F00D
:1050E0000EC008F00FC009F010C00AF0090ED890E9
:1050F0000736083609360A36E82E77EFA8F007504B
:10510000081009100A10D8B488EFA8F08BEFA8F0A7
:10511000010E8CEFA8F0000E036E046A94EFA8F065
:10512000000E046E040E036E120020EE13F0070E44
:10513000DE6AE806FDE20B500C100D100E100F1089
:10514000101011101210D8B4A8EFA8F0AAEFA8F010
:10515000FCEFA8F0010E1B6EB8EFA8F0D8900B364C
:105160000C360D360E360F361036113612361B2A17
:1051700012AEBDEFA8F0BFEFA8F0AEEFA8F0D89048
:1051800013361436153616361736183619361A36BB
:105190000B50035C0C5004580D5005580E50065827
:1051A0000F500758105008581150095812500A58FB
:1051B000D8A0DDEFA8F0DFEFA8F0F0EFA8F00B50DB
:1051C000035E0C50045A0D50055A0E50065A0F50EB
:1051D000075A1050085A1150095A12500A5A13808F
:1051E000D8901232113210320F320E320D320C3290
:1051F0000B321B2EBFEFA8F013C003F014C004F055
:1052000015C005F016C006F017C007F018C008F06A
:1052100019C009F01AC00AF0120005500610D8B4DF
:1052200014EFA9F016EFA9F01FEFA9F00550061032
:10523000D8A41DEFA9F01FEFA9F024EFA9F00350A7
:1052400043ECB8F078EFA9F020EE09F00550D9262C
:105250000650DA22DE50DE10D8B431EFA9F033EF79
:10526000A9F04EEFA9F020EE09F00550D92606501E
:10527000DA2210EE03F00550E1260650E222DE505D
:10528000E65CE650800A0B6EDE50800A0B58D8B000
:105290004CEFA9F04EEFA9F078EFA9F020EE03F063
:1052A0000550D9260650DA226F0078FF07F06F000C
:1052B00074FF08F0600017F0D9FF60001BF0DAFF00
:1052C0006F0078FF09F06F0074FF0AF0075009249F
:1052D000D96E08500A20DA6E60000FF0DFFF20EE72
:1052E00003F00550D9260650DA22DE2A000EDD2210
:1052F00012000B500C100D100E100F10101011108A
:105300001210D8B486EFA9F088EFA9F0D0EFA9F079
:10531000010E136E96EFA9F0D8900B360C360D36B1
:105320000E360F36103611361236132A12AE9BEF98
:10533000A9F09DEFA9F08CEFA9F00B50035C0C5085
:1053400004580D5005580E5006580F50075810506D
:1053500008581150095812500A58D8A0B2EFA9F0B5
:10536000B4EFA9F0C4EFA9F00B50035E0C50045A3F
:105370000D50055A0E50065A0F50075A1050085A31
:105380001150095A12500A5AD89012321132103262
:105390000F320E320D320C320B32132E9DEFA9F06C
:1053A00003C003F004C004F005C005F006C006F019
:1053B00007C007F008C008F009C009F00AC00AF0E9
:1053C0001200000EBA6EBB68040EBC6EEF0EC26E09
:1053D000C368A30EC46E000E3A01606F000E506FDA
:1053E000000E406F000E816F5169FC0E416FC00EC0
:1053F000616F000E006F000E016F000E026F000E55
:10540000036F000E046F000E086F000E096F000E90
:105410000A6F000E0B6F000E0C6F000E0D6F000E6A
:105420000E6F000E0F6F070E426F000E526F180EB8
:10543000626F436953696369446954696469080E1A
:10544000846F000E476F000E466F000E456F000E12
:10545000576F000E566F000E556F000E676F000EEF
:10546000666F000E656F000E126F210E136F220E15
:10547000146F000E156F130E166F170EE56F130ED7
:10548000E16F140EE26F1200270E0001FB6F81EF37
:10549000AAF0800EDEECAEF0DE0E216EF70E226E6C
:1054A0001EECB0F0800EDEECAEF09FEFAAF0C00E66
:1054B000DEECAEF0DE0E216EF70E226E1EECB0F0CA
:1054C000C00EDEECAEF09FEFAAF0940EDEECAEF074
:1054D000DE0E216EF70E226E1EECB0F0940EDEECA6
:1054E000AEF09FEFAAF0D40EDEECAEF0DE0E216E31
:1054F000F70E226E1EECB0F0D40EDEECAEF09FEF95
:10550000AAF026C028F027C029F02950000AD8B4F4
:105510008CEFAAF09FEFAAF02850010AD8B449EF07
:10552000AAF0030AD8B457EFAAF0010AD8B465EF7D
:10553000AAF0070AD8B473EFAAF09FEFAAF0D00E32
:10554000286ECA0EE82EFED7282EFCD712000001C6
:10555000EAA1ADEFAAF0AFEFAAF0B9EFAAF015C03B
:105560000CF016C00DF013C00EF014C00FF0BDEC1F
:10557000B4F018BEBEEFAAF0C0EFAAF0C6EFAAF0D2
:1055800017C01CF018C01DF0CAEFAAF0000E1D6E67
:10559000000E1C6E000E1B6E000E1A6EDCEFAAF0E1
:1055A000000E046E200E036E13C005F014C006F04A
:1055B0000DECA9F01A4A1B2A1C501A5C1B50800AD9
:1055C000196E1D50800A1958D8A0E9EFAAF0EBEF28
:1055D000AAF0D0EFAAF00001EAB1F1EFAAF0F3EFE0
:1055E000AAF0FDEFAAF015C00CF016C00DF013C024
:1055F0000EF014C00FF0BDECB4F015C003F016C0EF
:1056000004F09DECB2F01C500324136E1D500420D6
:10561000146E1200000E086E06BE13EFABF011EF11
:10562000ABF019EFABF0056C061ED8B0062A010EE0
:10563000086E04BE20EFABF01EEFABF026EFABF030
:10564000036C041ED8B0042A010E081A000E0A6E5C
:10565000000E096E05500610D8B431EFABF033EFF1
:10566000ABF05BEFABF0010E076E3BEFABF0D89009
:1056700005360636072A06AE40EFABF042EFABF038
:1056800037EFABF0D89009360A360550035C065068
:105690000458D8A04EEFABF050EFABF055EFABF0A5
:1056A0000550035E0650045A0980D8900632053230
:1056B000072E42EFABF00850D8B461EFABF063EFC8
:1056C000ABF067EFABF0096C0A1ED8B00A2A09C02C
:1056D00003F00AC004F01200000E086E04BE75EF5D
:1056E000ABF073EFABF07BEFABF0036C041ED8B004
:1056F000042A010E086E06BE82EFABF080EFABF01D
:1057000086EFABF0056C061ED8B0062A05500610D1
:10571000D8B48DEFABF08FEFABF0B3EFABF0010E81
:10572000076E97EFABF0D89005360636072A06AE1F
:105730009CEFABF09EEFABF093EFABF00550035C4A
:1057400006500458D8A0A7EFABF0A9EFABF0ADEF2F
:10575000ABF00550035E0650045AD890063205326D
:10576000072E9EEFABF00850D8B4B9EFABF0BBEF0B
:10577000ABF0BFEFABF0036C041ED8B0042A03C03B
:1057800003F004C004F01200D40EF66E670EF76E3C
:10579000010EF86E00EEA8F210EE48F009006F005E
:1057A000D7FFEEFFE550E150F9E1A60EF66E6D0E63
:1057B000F76E010EF86E00EED5F110EE26F009003E
:1057C0006F00D7FFEEFFE550E150F9E1840EF66E71
:1057D000700EF76E010EF86E09006F00D4FF5CF0DA
:1057E00009006F00D4FF5DF001EE00F0800EEE6A5C
:1057F000E806FDE100EE00F3A00EEE6AE806FDE12A
:1058000000EE00F2A80EEE6AE806FDE100EE00F1FF
:10581000D50EEE6AE806FDE100EEE8F0170EEE6A3E
:10582000E806FDE1080ED56E000ED66E000ED76EAE
:10583000000107EF86F0000E03140B6E000E041437
:105840000C6E800E05140D6E7F0E06140E6E0B503E
:105850000C100D100E10D8A430EFACF032EFACF0FD
:105860003AEFACF0000E036E000E046E000E056EF3
:10587000000E066E000E07140B6E000E08140C6E60
:10588000800E09140D6E7F0E0A140E6E0B500C1054
:105890000D100E10D8A44FEFACF051EFACF059EF53
:1058A000ACF0000E076E000E086E000E096E000EC2
:1058B0000A6E075003180FE1085004180CE1095054
:1058C000051809E10A500618D8B469EFACF06BEF7F
:1058D000ACF06EEFACF0D8906FEFACF0D880120067
:1058E000266E270E0001FB6F2250236E246A235080
:1058F0005C5C5D50800A256E2450800A2558D8B023
:1059000084EFACF086EFACF088EFACF05C04226E74
:105910002604D8A48EEFACF090EFACF094EFACF08E
:1059200022507F0FDEECAEF0020E2618D8A49BEFBB
:10593000ACF09DEFACF0A1EFACF02250BF0FDEEC6D
:10594000AEF0030E2618D8A4A8EFACF0AAEFACF086
:10595000AEEFACF02250930FDEECAEF0040E261842
:10596000D8A4B5EFACF0B7EFACF0BBEFACF0225081
:10597000D30FDEECAEF0D00E236ECA0EE82EFED7AB
:10598000232EFCD71200036E010E046E010129B70D
:10599000CCEFACF0CEEFACF013EFADF003C022F1E2
:1059A00029952987FC0E29170F0E276F010E216FED
:1059B000F40E206F2989800E006F700E016F010EAA
:1059C000026F000E126F000E136F800E036F700EC9
:1059D000046F010E056F000E146F000E156F800E20
:1059E000066F700E076F010E086F000E166F000E27
:1059F000176F800E096F700E0A6F010E0B6F000E8D
:105A0000186F000E196F7C0E0C6F700E0D6F010E6B
:105A10000E6F000E1A6F000E1B6F18ECB8F03BEC07
:105A2000B6F0000E046E045012000101298939EF0E
:105A3000ADF02BECB8F0080E66EFADF02BECB8F043
:105A4000070E66EFADF001012529FEECB7F0040E5C
:105A500066EFADF0070E01012719D8B432EFADF0B3
:105A600034EFADF036EFADF02EECB8F00F0E66EF80
:105A7000ADF012C10EF013C10FF002D84AEFADF035
:105A80000500FA6E0051FD6E0151FE6E0251FF6E6F
:105A9000FA501200106E116A1150000AD8B453EF78
:105AA000ADF02AEFADF01050010AD8B42AEFADF0F6
:105AB000030AD8B41EEFADF0010AD8B419EFADF067
:0E5AC000070AD8B423EFADF02AEFADF01200C4
:105AD0003901A3A76EEFADF070EFADF0B7EFADF009
:105AE00093A775EFADF077EFADF0B7EFADF06F00C6
:105AF000A0F7BFF10D0E0101BF19D8B482EFADF0D0
:105B000084EFADF090EFADF00001F35109E1800EAC
:105B1000F25DD8A08EEFADF090EFADF0A8EFADF054
:105B2000010E0101C06F200E0001F225D96E030E97
:105B3000F321DA6E000EDF6EF2C0F6F0F3C0F7F07C
:105B4000000EF36F000EF26F39019397B7EFADF0CF
:105B5000200EF225D96E030EF321DA6E6000FFF6F7
:105B6000DFFFF24BF32BF2C0F6F0F3C0F7F01100B9
:105B70009AECB7F00009D8A4C0EFADF0C2EFADF0D9
:105B8000C5EFADF0040E06EFAEF001012951030B95
:105B90000009D8B4CEEFADF0D0EFADF0DCEFADF052
:105BA000010E126E2951030B136E1250135E295110
:105BB0001318FC0B1318296F2507D8A026072551A9
:105BC0002611D8B4E6EFADF0E8EFADF0F6EFADF0AA
:105BD00028ECB8F060008FF4D9FF600093F4DAFF8E
:105BE000DF6E0101234B242BC2EFADF015ECADF0BD
:105BF000146E28ECB8F060008FF4D9FF600093F4C5
:105C0000DAFFDF6E0101234B242B14501200216EAA
:105C1000270E0001FB6F2150F00B0C09226E22C0F1
:105C20001DF0FB5169ECB6F02A0EE82EFED700D02D
:105C30002150F00B0809226E22C01DF00001FB511B
:105C400069ECB6F02A0EE82EFED700D01F04D8A4C7
:105C50002CEFAEF02EEFAEF052EFAEF021C020F000
:105C60000F0E20162038F00B0C09226E22C01DF0FA
:105C70000001FB5169ECB6F02A0EE82EFED700D0E9
:105C800021C020F00F0E20162038F00B0809226EDC
:105C900022C01DF00001FB5169ECB6F02A0EE82E7F
:105CA000FED700D01200086E035004100510D8B4BF
:105CB0005CEFAEF05EEFAEF07FEFAEF00850030D9C
:105CC000000EF324D96E010EF420DA6E60000FF09E
:105CD000DEFF600013F0DEFF600017F0DEFF08500B
:105CE000020D120EF324D96E010EF420DA6E60005C
:105CF0001BF0DEFF60001FF0DDFF99EFAEF00850F3
:105D0000030D000EF324D96E010EF420DA6E800E1E
:105D1000DE6E700EDE6E010EDE6E0850020D120E8B
:105D2000F324D96E010EF420DA6E000EDE6E000E42
:105D3000DD6E1200206E270E0001FB6F2050F00B6D
:105D40000D09FA6FFAC01DF0FB5169ECB6F02A0E8E
:105D5000E82EFED700D02050F00B09090001FA6FA1
:105D6000FAC01DF0FB5169ECB6F02A0EE82EFED702
:105D700000D020C01FF00F0E1F161F38F00B0D09AA
:105D80000001FA6FFAC01DF0FB5169ECB6F02A0E63
:105D9000E82EFED700D020C01FF00F0E1F161F38B0
:105DA000F00B09090001FA6FFAC01DF0FB5169EC14
:105DB000B6F02A0EE82EFED700D01200206E270E75
:105DC0000001FB6F2050F00B0C09216E21C01DF06B
:105DD000FB5169ECB6F02A0EE82EFED700D0205019
:105DE000F00B0809216E21C01DF00001FB5169EC88
:105DF000B6F06A0EE82EFED700D020C01FF00F0EBE
:105E00001F161F38F00B0C09216E21C01DF0000178
:105E1000FB5169ECB6F06A0EE82EFED700D020C028
:105E20001FF00F0E1F161F38F00B0809216E21C03E
:105E30001DF00001FB5169ECB6F06A0EE82EFED7AA
:105E400000D012001D6E19C020F01AC021F01BC036
:105E50001EF01CC01FF01D50C3ECACF00009D8B4FC
:105E600034EFAFF036EFAFF02BEFAFF0840E096EEA
:105E7000670E0A6E010E0B6E1E0E0C6E000E0D6E7E
:105E80006BECB7F0180E036E000E046E000E066E7B
:105E9000010E056E0BECB7F0000E096E000E0A6ED7
:105EA000000E0B6E000E0C6E000E0D6E5DECB7F06A
:105EB00008ECB8F07FECB6F0E806D8B462EFAFF0CB
:105EC00064EFAFF05AEFAFF01200010129897AEFC9
:105ED000AFF02BECB8F0070EA3EFAFF001012529CE
:105EE000FEECB7F0030EA3EFAFF02EECB8F00A0E05
:105EF000A3EFAFF012C10EF013C10FF002D88BEF79
:105F0000AFF00500FA6E0051FD6E0151FE6E0251B8
:105F1000FF6EFA501200106E116A1150000AD8B4C8
:105F200094EFAFF075EFAFF01050010AD8B475EFF1
:105F3000AFF0030AD8B469EFAFF0060AD8B46EEF39
:105F4000AFF075EFAFF012003901949BA49BC4949D
:105F5000260E3A01126F3F013E9F3E9F000E3E6F9C
:105F6000030E3F6F000E3A6F000E396F000E386F50
:105F7000630E0101D16F100ED26F000ED36F000EB1
:105F8000D46FD10E6E6F010E6F6F20EE02F06E5166
:105F9000D9266F51DA22DF503F013D6F010120EE1B
:105FA00001F06E51D9266F51DA22DF503F013C6F6C
:105FB0006000BBF5D9FF6000BFF5DAFFDF503B6F33
:105FC0003E8F12003901A3A7E8EFAFF0EAEFAFF080
:105FD000EDEFAFF06F00A0F7BFF1000E046E000E02
:105FE000036E200E0324D96E030E0420DA6E000E19
:105FF000DF6E034A042A045009E17F0E035CD8A037
:1060000004EFB0F006EFB0F0F1EFAFF0000E0101D9
:10601000C06F3D01F289000EF96F000EFA6F000E9D
:106020000301206F000E0001F76F000EF66F000EE7
:106030000101BF6F3901938D93871200000E256E09
:10604000000E246E38EFB0F0600087F0F6FF6000BD
:106050008BF0F7FF000EF86E0800F5509AECAEF0EA
:10606000214A222A244A252A850EE82EFED700F04E
:10607000600087F0F6FF60008BF0F7FF000EF86E0F
:106080000800F5500009D8B448EFB0F04AEFB0F07E
:1060900059EFB0F05C50245C2550800A236E5D50AF
:1060A000800A2358D8A057EFB0F059EFB0F024EF92
:1060B000B0F0120018ECB8F0020E0101286F6DEF7D
:1060C000B0F0E6ECB7F094EFB0F03CECB8F094EF41
:1060D000B0F0D7ECB7F094EFB0F014C10EF015C1EA
:1060E0000FF020EE03F102D880EFB0F00500FA6E59
:1060F000DE50FD6EDE50FE6EDE50FF6EFA50120076
:10610000106E116A1150000AD8B489EFB0F069EF2F
:10611000B0F01050020AD8B461EFB0F0010AD8B460
:1061200065EFB0F069EFB0F01200C3C0C7F0C4C0B3
:10613000C8F0000E0101676F000E666FB7EFB0F098
:10614000C1C099F0C2C09AF0C70E00019B6F000E4B
:106150009C6FC5C09DF0C6C09EF0E0EC8BF00001C6
:1061600099510101662700019A51010167236000DE
:106170001FF3F6FF600023F3F7FF000EF86E080030
:10618000F5500009D8A4C7EFB0F0C9EFB0F0A0EF08
:10619000B0F066C1C1F067C1C2F01200600017F034
:1061A000F6FF60001BF0F7FF000EF86E08006F00AE
:1061B000D4FFBEF1F5EFB0F0600017F0F6FF60001D
:1061C0001BF0F7FF000EF86E08006F00D4FFBEF161
:1061D00060000FF0D9FF600013F0DAFF6000FBF6FB
:1061E000DFFF034A042A054A062A0101BE51D8A44A
:1061F000FCEFB0F0FEEFB0F0DCEFB0F060000FF0BD
:10620000D9FF600013F0DAFF000EDF6E120099EC88
:10621000B3F001012951030B0009D8B412EFB1F01A
:1062200014EFB1F021EFB1F08FECB7F00009D8B462
:106230001CEFB1F01EEFB1F021EFB1F0100E010133
:10624000276F01012751030D470EF324F66EF50E5B
:10625000F420F76EF86A000EF82202D83DEFB1F094
:106260000500FA6E0900F550FD6E0900F550FE6E4E
:106270000900F550FF6EFA5012000101276F12005D
:10628000000E066E000E056E69EFB1F03901A3A98C
:106290004CEFB1F04EEFB1F046EFB1F005500324F2
:1062A000D96E06500420DA6EDF503D01EA6F054AD0
:1062B000062A06BE65EFB1F0065009E1810E055CC5
:1062C000D8A065EFB1F067EFB1F069EFB1F077EF0B
:1062D000B1F005500324D96E06500420DA6EDF5069
:1062E000D8A475EFB1F077EFB1F046EFB1F012003E
:1062F000FC0E01012917020E286F299587EFB1F0D6
:106300003AECB8F0AEEFB1F00F0EAEEFB1F016C14F
:106310000EF017C10FF020EE06F102D89AEFB1F09F
:106320000500FA6EDE50FD6EDE50FE6EDE50FF6E32
:10633000FA501200106E116A1150000AD8B4A3EF7F
:10634000B1F084EFB1F01050020AD8B480EFB1F090
:10635000010AD8B480EFB1F084EFB1F0120009C0A7
:106360000DF00AC00EF007C00FF008C010F00D507D
:106370000B6E0E500C6E0D4A0E2A60002FF0F6FFC9
:10638000600033F0F7FF000EF86E60003FF0D9FFB9
:10639000600043F0DAFF0F4A102A1F0EF76403D0A3
:1063A0000800F55007D06F00DBFFE9FF6F00DFFF4B
:1063B000EAFFEF50DF6EDF50D8A4E1EFB1F0E3EF7A
:1063C000B1F0B7EFB1F01200000E256E000E246E92
:1063D000F5EFB1F024502124D96E25502220DA6E39
:1063E000DF509AECAEF0244A252A24502124D96E9D
:1063F00025502220DA6EDF50D8B401EFB2F003EF5F
:10640000B2F012EFB2F05C50245C2550800A236E8B
:106410005D50800A2358D8A010EFB2F012EFB2F00E
:10642000EAEFB1F012001C6E1C50C3ECACF0000996
:10643000D8B41DEFB2F01FEFB2F014EFB2F018C0F5
:1064400003F019C004F01AC005F01BC006F00BECF5
:10645000B7F0000E096E000E0A6E000E0B6E000EF5
:106460000C6E000E0D6E5DECB7F008ECB8F07FEC32
:10647000B6F0E806D8B43FEFB2F041EFB2F037EF34
:10648000B2F012003901A3A148EFB2F04AEFB2F026
:106490004CEFB2F06FEFB2F0A2AF51EFB2F053EFAA
:1064A000B2F055EFB2F06FEFB2F03D0179A55BEFBE
:1064B000B2F05DEFB2F05FEFB2F06FEFB2F079AF34
:1064C00064EFB2F066EFB2F068EFB2F06FEFB2F0E7
:1064D00076A96DEFB2F06FEFB2F042EFB2F01200BA
:1064E000D28AD2BE76EFB2F079EFB2F0010E7AEF37
:1064F000B2F0000E036ED29ED29CD28A550ED46E9C
:10650000AA0ED46ED490000ED76E000ED66E080E72
:10651000D56E550ED46EAA0ED46ED4803901838701
:10652000828F81818491839F84858791899103B033
:1065300002D0D29E01D0D28E120003C005F004C05A
:1065400006F0A5EFB2F0034A042A60000FF0F6FF50
:10655000600013F0F7FF000EF86E1F0EF76403D013
:106560000800F55007D06F00DBFFE9FF6F00DFFF89
:10657000EAFFEF500009D8A4C0EFB2F0C2EFB2F0CA
:10658000A3EFB2F00550035C036E06500458046E8E
:106590001200E1EFB2F03901A3A9D1EFB2F0D3EFCD
:1065A000B2F0CBEFB2F060000FF0F6FF600013F036
:1065B000F7FF000EF86E08006F00D7FFEAFD034AF0
:1065C000042A60000FF0F6FF600013F0F7FF000EE2
:1065D000F86E0800F5500009D8A4F1EFB2F0F3EF1F
:1065E000B2F0CBEFB2F01200066E000E01016D6F3B
:1065F000000E6C6F0BEFB3F0520E046E2B0E036E99
:10660000000EE82EFED7032EFCD7042EFAD700D0BA
:1066100001016C4B6D2B0650036E046A03506C5DD8
:106620006D51800A056E0450800A0558D8A01BEFF2
:10663000B3F01DEFB3F0FCEFB2F01200CD0E00018D
:10664000D56F000ED66FC9C0D7F0CAC0D8F0000E03
:10665000DB6F000EDA6F000EE16F000EE06FD70EF9
:10666000C16F000EC26FCBC0C3F0CCC0C4F0D50E5A
:10667000C56F000EC66F95ECB0F00001DA51C92568
:10668000D96EDB51CA21DA6E000EDF6E1200010EE8
:10669000096E200E03180410D8B451EFB3F053EF75
:1066A000B3F06CEFB3F0F70E056EFF0E066E03C08D
:1066B00007F004C008F005500726065008220850CD
:1066C00009E1050E075CD8A068EFB3F06AEFB3F0FC
:1066D0006CEFB3F0000E096E09C003F0046A1200FB
:1066E000166E010E176E010129B579EFB3F07BEF3D
:1066F000B3F097EFB3F02985000E176E2551FEEC2D
:10670000B7F01650D8B487EFB3F089EFB3F090EF3D
:10671000B3F0040E0101276F52ECB6F095EFB3F021
:10672000030E0101276F79ECB7F03FECB7F017507B
:106730001200BBECB7F00009D8B4A1EFB3F0A3EF9F
:10674000B3F0A7EFB3F037ECB8F0C1EFB3F0A5ECBE
:10675000B7F00009D8B4AFEFB3F0B1EFB3F0B5EFD5
:10676000B3F031ECB8F0C1EFB3F0B0ECB7F0000922
:10677000D8B4BDEFB3F0BFEFB3F0C1EFB3F034EC7A
:10678000B8F0120020EE02F00E50D9260F50DA2297
:106790006F0078FF03F06F0074FF04F060003BF0BF
:1067A000D9FF60003FF0DAFF6F0078FF05F06F005F
:1067B00074FF06F00BECB7F0000E096E000E0A6EC7
:1067C000000E0B6E000E0C6E000E0D6E6BECB7F033
:1067D000020E120083F872F869F8BAF8A7F8C6F842
:1067E000B4F860F8AEF805F857F843F839F84DF703
:1067F000F4F524F795F776F79DF5F3F77AF6BAF600
:10680000F1F6A0F899F892F82FF88BF825F87BF8B4
:106810001BF8C0F810F84DF8B4F7C9F7000E3D01A9
:10682000EC6F000EED6F000EEE6F000EEF6F000EBE
:10683000F06F000EF16FB00EF26F800EF36F000E6E
:10684000F46F8A0EF56F000EF66F000EF76F000EF4
:10685000F86F000EF96F000EFA6FF28BF2893901B2
:1068600093971200046E800E056E4CEFB4F0045046
:1068700005140009D8B43FEFB4F041EFB4F046EF8F
:10688000B4F02A0E2FECB7F049EFB4F0200E2FEC45
:10689000B7F0D8900530056E0550D8A452EFB4F08B
:1068A00054EFB4F037EFB4F01200BF0E0B6EFF0ED2
:1068B0000C6E09C00DF00AC00EF00B500D260C50E6
:1068C0000E220E5007E11A0E0D5CD8B06AEFB4F03C
:1068D0006CEFB4F073EFB4F0200E0910096E0A509B
:1068E0000A6E77EFB4F009C009F00AC00AF012008E
:1068F000000E2E1A000E2F1A000E301A800E311ABA
:106900002AC003F02BC004F02CC005F02DC006F007
:106910002EC007F02FC008F030C009F031C00AF0D7
:1069200080EC91F003C02AF004C02BF005C02CF0DD
:1069300006C02DF012009F0E0B6EFF0E0C6E09C0EC
:106940000DF00AC00EF00B500D260C500E220E500A
:1069500007E11A0E0D5CD8B0B0EFB4F0B2EFB4F0AE
:10696000B8EFB4F05F0E0914096E0A6ABCEFB4F018
:1069700009C009F00AC00AF01200000E126E000EE3
:10698000116ECEEFB4F010C003F0046A0EC005F033
:106990000FC006F00DECA9F0114A122A11500C2478
:1069A000D96E12500D20DA6EDF50106E1050D8A440
:1069B000DCEFB4F0DEEFB4F0C3EFB4F0120016BEBB
:1069C000ECEFB4F0165006E11504D8B0EAEFB4F0DD
:1069D000ECEFB4F0FAEFB4F015C017F016C018F0F1
:1069E000171E181E174A182A17C015F018C016F0DF
:1069F000FEEFB4F015C015F016C016F012009F0E91
:106A0000056EFF0E066E200E0310076E000E0410BA
:106A1000086E055007260650082208500AE11A0E93
:106A2000075CD8A016EFB5F019EFB5F0010E1AEF1C
:106A3000B5F0000E036E046A12009F0E056EFF0E85
:106A4000066E03C007F004C008F005500726065084
:106A5000082208500AE11A0E075CD8A032EFB5F000
:106A600035EFB5F0010E36EFB5F0000E036E046A97
:106A70001200BF0E056EFF0E066E03C007F004C0C5
:106A800008F0055007260650082208500AE11A0EA1
:106A9000075CD8A04EEFB5F051EFB5F0010E52EF04
:106AA000B5F0000E036E046A1200035004100510C6
:106AB0000610D8B45EEFB5F060EFB5F068EFB5F052
:106AC000000E031A000E041A000E051A800E061A94
:106AD00003C003F004C004F005C005F006C006F0D2
:106AE0001200D00E056EFF0E066E03C007F004C044
:106AF00008F0055007260650082208500AE10A0E41
:106B0000075CD8A086EFB5F089EFB5F0010E8AEFEB
:0A6B1000B5F0000E036E046A1200D7
:106B1C006F0060FF02F001017C4B7D2B000E896F32
:106B2C00010E886F7D5109E1050E7C5DD8A0A1EFA7
:106B3C00B5F0A3EFB5F0A4EFB5F0B4853901A49589
:106B4C0060000BF0D8FF1100036E3D0179956000D9
:106B5C000FF06EFD000E6C6F738B79A5B8EFB5F06E
:106B6C00BAEFB5F0B3EFB5F074ABBFEFB5F0C2EF61
:106B7C00B5F0010EC3EFB5F0000E12000EC003F01D
:106B8C000FC004F0000E066E010E056E0BECB7F094
:106B9C00000E096E000E0A6E000E0B6E000E0C6ECF
:106BAC00000E0D6E6BECB7F0040E12000EC003F06D
:106BBC000FC004F0000E066E020E056E0BECB7F063
:106BCC00000E096E000E0A6E000E0B6E000E0C6E9F
:106BDC00000E0D6E6BECB7F0020E12000EC003F03F
:106BEC000FC004F0000E066E010E056E0BECB7F034
:106BFC00000E096E000E0A6E000E0B6E000E0C6E6F
:106C0C00000E0D6E6BECB7F0020E12000EC003F00E
:106C1C000FC004F0000E066E020E056E0BECB7F002
:106C2C00000E096E000E0A6E000E0B6E000E0C6E3E
:106C3C00000E0D6E6BECB7F0040E12003901A3A917
:106C4C002AEFB6F02CEFB6F024EFB6F00D0E3D01A6
:106C5C00EA6F3901A3A935EFB6F037EFB6F02FEF95
:106C6C00B6F00A0E3D01EA6F12003D0173BF41EF11
:106C7C00B6F043EFB6F051EFB6F0000E796F000EA0
:106C8C007A6F000E766F6C69510E3A016A6F510E75
:106C9C006B6F3D01738F120001012951FC0B02092E
:106CAC00296F25052611D8A45EEFB6F060EFB6F07B
:106CBC0062EFB6F015ECADF0D88001012235F9EC9D
:106CCC00B7F0040E12001E6E1DC0C1F1000E0101C2
:106CDC00C26FC10E186E010E196E000E1B6E010EE6
:106CEC001A6E1E5013ECB2F0A00E00D0E82EFDD799
:106CFC001200010E036E010129B587EFB6F089EF82
:106D0C00B6F093EFB6F02997226918ECB8F04EEC78
:106D1C00B7F0F3ECB7F028C103F0035012000350A6
:106D2C0005026F00CCFF07F06F00D0FF08F0035096
:106D3C000602F350082604500502F350082607C03B
:106D4C0003F008C004F012002B6E27C022F02B5069
:106D5C0070ECACF028C021F029C022F0E4ECB1F0CA
:106D6C00150E2A6EC60EE82EFED72A2EFCD700D0A2
:106D7C0012001FECB8F01CECB8F00009D8B4C9EF45
:106D8C00B6F0CBEFB6F0D1EFB6F0000EFEECB7F0EC
:106D9C00000EF9ECB7F0000E1200286E756C6C2921
:106DAC000001000200040008001000008030304890
:106DBC0030304D3030530030302F30302F303000E9
:106DCC0011C003F012C004F09DECB2F0035011247A
:106DDC00076E04501220086E13C009F014C00AF09C
:106DEC00AFECB1F01200030E3D017B6F040E736F1C
:106DFC00800E746F000E756F000E6C6F75996000CD
:106E0C00EFF36EFD7995739F1200010129A911EF23
:106E1C00B7F013EFB7F01CEFB7F003C023F104C0C9
:0E6E2C0024F105C025F106C026F129991200B7
:106E3C006F0060FF01F001018E4B8F2BB481660E49
:106E4C00B76E7C0EB66E3901A39F600007F0D8FFB9
:106E5C001100036E33EFB7F000F03901A3A939EF3D
:106E6C00B7F03BEFB7F032EFB7F060000FF0EAFD90
:106E7C00120045EFB7F042ECB2F007ECB1F00101B3
:106E8C0029B54BEFB7F04DEFB7F041EFB7F012006B
:106E9C00390193939395929F93913D017A917A95B1
:106EAC007A9F7A9D7A93769376957691120009C0A3
:106EBC0003F00AC004F00BC005F00CC006F00DC0C6
:106ECC0007F0020E53ECAEF0120009C003F00AC03A
:106EDC0004F00BC005F00CC006F00DC007F0000E5E
:106EEC0053ECAEF0120001012951FC0B0209296F81
:106EFC0022512225F9ECB7F0030E12003D0178BBAC
:106F0C008AEFB7F08DEFB7F0010E8EEFB7F0000EF1
:106F1C0012003D0174BB95EFB7F098EFB7F0010E7E
:106F2C0099EFB7F0000E12003D0178B1A0EFB7F069
:106F3C00A3EFB7F0010EA4EFB7F0000E12003D0165
:106F4C0079B5ABEFB7F0AEEFB7F0010EAFEFB7F02E
:106F5C00000E12003D0176B9B6EFB7F0B9EFB7F0FD
:106F6C00010EBAEFB7F0000E12003D0179BFC1EF70
:106F7C00B7F0C4EFB7F0010EC5EFB7F0000E12007A
:106F8C000101904B912B3F013E8FC4943901A1918B
:106F9C00110003ECB8F001012995020E286F0F0EB9
:106FAC00120003ECB8F001012995000E286F0F0EAA
:106FBC00120022ECB8F01FECB8F0EDECB7F01200B8
:106FCC0001012551FEECB7F052ECB6F012000101B4
:106FDC002995000E286F0F0E12003D01739F000EB5
:106FEC00796F78851200036E60000FF06BFD120054
:106FFC00036E60000FF06CFD12003D01739F7885ED
:10700C00738F1200000E70ECB3F0120022ECB8F08B
:10701C00090E120025ECB8F0040E120025ECB8F0A5
:10702C00030E1200000E3D01796F12003D016C51F0
:10703C0012003D01739B12003D01748D12003D0145
:10704C00749D12003D016A5112003D01738D1200B6
:10705C003D01739D12003D01799512003D01769919
:10706C0012003D01799F1200010E1200020E120057
:0C707C00050E1200010E1200140012009C
:020000040030CA
:0A0000008CD5FFF78DCFFFDFFFFF67
:00000001FF
